:100000000C94960A0C94DD0A0C94DD0A0C94DD0A1B
:100010000C94DD0A0C94DD0A0C94DD0A0C94DD0AC4
:100020000C94DD0A0C94DD0A0C940C300C94DB303B
:100030000C9490290C94DD0A0C94DD0A0C94DD0AD2
:100040000C94DD0A0C94DD0A0C94DD0A0C94DD0A94
:100050000C94DD0A0C94E9290C94DD0A0C94DD0A59
:100060000C94DD0A0C94DD0A0C94DD0A0C94DD0A74
:100070000C94DD0A0C94DD0A0C94DD0A0C94DD0A64
:100080000C94DD0A0C94DD0A0C94DD0A0C94DD0A54
:100090000C94DD0A0C94DD0A0C94DD0A0C94DD0A44
:1000A0000C94DD0A0C94DD0A0C94DD0A5A185D18D4
:1000B0006F18801888189318EA18EA18EA18D818E0
:1000C000DB18961899189D18AA18B718BA18BE18F0
:1000D000CB180C200C203E203E208B20B221B221D8
:1000E000B221A9204221532153214E224E226022C7
:1000F000602257226022602260224E224E225C2221
:10010000602260225C2248316F3167326F31673282
:10011000BB31DE316732353244320A0062757273A8
:1001200074206F6E00256325632563256325632591
:1001300063256325637C0001048E966E773EFE7E08
:100140005F1DB8F2664EFF5D19B0C20469542AD62D
:100150002EBFDD19B0C3E529B1E023A5A9B1C100C7
:1001600082674C1A978D795120C7068E7C7C7A76EF
:100170004FFD5930E2460E9EBEDF1D9991A0A5A10C
:10018000A9D022C6EF5C1B958990A2A7CCFB55286D
:10019000B3E44AF76C3BF46A562EDE1F9DB8D305D4
:1001A0008892A6CE1EBEDF1D99B0E246EF5C071115
:1001B0005D980B9D9497EE4E45336B44C7295627A7
:1001C00030C6A7D5F256DFB43862CBA0B6E30F84B1
:1001D000062405656F7689B577412782666582CCEE
:1001E000D5E620D52717C5F803237C5F64A51DC17C
:1001F000D636CB4CD4DB66D78BB1997E6F4C36406C
:1002000006D6EBD7A2E4F495515A5496D55344D769
:100210008CE0B94068D218E9DD9A239248EE7F431A
:10022000AFEA7738848C0A72AF69F8DDF12483A3D2
:10023000F84ABFF59413DBBBD8B4B3A0FB455060BC
:100240003059123171A2D313E7FAE7CE0F63150BC1
:100250006B94BB378326059DFB4692FC0A15D10D96
:100260007392D68C1B8CB8558ACEBDFE8EFCED09E0
:1002700012839182513123FBB40C76AD7CD9B44BFF
:10028000B26714099C7F0C18BA3BD68E142AE41B63
:10029000529F2B7DE1FB6A3302FAAC5AF23E887E14
:1002A000AED1F378E805D1E3DC21F6E19ABD170E73
:1002B000D9469B8803EAF666BE0E1B5049964097C6
:1002C000F1F1E480A66EE87734BF294044C2FF4EC6
:1002D00098D39CA3322B76510409E7A9D1A632B159
:1002E0002353E247ABD6F5695C3E5FFAAE4520E5A5
:1002F000D244FF39326DFD27575CFDF0DEC1B59960
:10030000E5F51C770175C56D5892F2B247000126DC
:10031000967A30FFB7F0EF77C18A5DDCC0D1293023
:100320001E77387A94F1B87A7EEFA4D1AC314AF2D4
:100330005D643DB2E2F00899FC70EE24A77EEE1EEB
:1003400020697D44BF8742DF883B0CDA42C904F94B
:100350004550FC838F116A72BC9995F0AC3DA73B68
:10036000CD1CE2887937115F3989950A16847AF6AF
:100370008AA428E4ED83803BB123A50310F466EA48
:10038000BB0C0FC5EC6C69C5D324ABD42AB79988D4
:100390007608A0A8957CD8386DCD5902514BF1B59F
:1003A0002B50E3B6BDD072CF9EFD6EBB44C8248AED
:1003B00077188A1306EF977DFA81F031E6FA77ED28
:1003C0003106315B548A9F3068DBE240F84E73FAA5
:1003D000AB748B105813DCD2E678D1322E8A9F2C66
:1003E00058064827C5A95E8147894621910370A414
:1003F0003E889CDA330ACEBC8B8ECF9FD37180436C
:10040000CF6BA95183763082C56A853911501A8223
:10041000DC1E1CD57DA9719933471997B35AB1DFFA
:10042000EDA4F2E62684A2289A9EDFA66AF4D6FC02
:100430002E5B9D1A2A2768FBC183214B90E036DD95
:100440005B314255A013F7D089537199570929C5DB
:10045000F321F8372F40F3D4AF16083602FC77C5E6
:100460008B049056B9C9679A99E800D386FF972DF7
:1004700008E9B7B391BCDF45C6ED0F8C4C1EE65BB7
:100480006E3830E4AAE395DEB9E49AF5B2559A875E
:100490009BF66AB2F2779A31F47A31D11D04C07CAE
:1004A00032A29E9AF562F8278DBF51FFD3DF6437E1
:1004B0003F2A6F763A7D77069E777F5EEB3251F961
:1004C00016669A09F3B008A470964630FFDA4FE931
:1004D0001BED8DF8741F3192B3731736DB9130D654
:1004E00088556B3477877AE7EE06C61C8C190C4862
:1004F00046235E9C075CBFB47ED64F749CE2C55019
:100500008BC58B159060625729D01343A1808891C9
:100510000044C74D1986CC2F2A755AFCEB972A70D8
:10052000E378D891B04F9907A395EA2421D5DE51FD
:100530002093270A3073A8FF8A97E9A76A8E0DE8EF
:10054000F0DFECEAB46C1D392A622D3D5A8B65F858
:1005500090052E7E912C78EF8E7AC12FAC78EEAF7D
:100560002845064C26AF3BA2DBA39306B53CA5D895
:10057000EE8FAF25CC3F856848A962CC978F7F2A44
:10058000EAE0150AAD6207BD45F841D836CB4CDB31
:100590006EE63AE7DA15E9291E1210A0142C0E3D7A
:1005A000F4BF394192750B257BA3CE399C1564C8E5
:1005B000FA3DEF7327FE262ECEDA6EFD718EDDFE3C
:1005C00076EEDC125C02C53A4E4E4FBFCA4015C7EC
:1005D0006E8D41F110E04F7E977F1CAE478E6BB160
:1005E0002531B073C71B9779F980D3662230077421
:1005F0001EE4D08021D6EE6B6C4FBFF5B7D90987CA
:100600002FA914BE27D9725001D41373A6A7510283
:100610007525E1B345347DA88EEBF31649CB4F8C9D
:10062000A1B9368539755D0800AEEBF6EAD7133A05
:10063000215A5F3084522695C914F257556BB11078
:10064000C2E1BD3B51C0B7554C711226C70DF951DF
:10065000A43802057FB8F1724BBF718914F3773863
:10066000D97124F30011A1D8D46927083735C911ED
:100670009D901C0EE71CFF2D1EE892E11810957C42
:10068000E080F4964321F975216438DD9F1E9516AC
:10069000DA561D4F9A53B2E2E418CB6B1A65EB564B
:1006A000C63BE5FED8263F3A84597266A2F375FF31
:1006B000FB60B322AD3F2D6BF9EBEA057CD88F6D63
:1006C0002C989E2B93F15E46F08749297368D77F5B
:1006D000F9F0E57DDB1D7519F3C4589B1788A892C6
:1006E000E0BEBD8B1D8D9F5676ADAF29E2D9D552A8
:1006F000F6B55635573AC8E156431994D3049B6D65
:1007000035D80B5F4D198EECFA64910A72202BBC20
:100710001A4AFE8BFDBBED1B23EAAD7282A129991B
:1007200071BDF095C103DD7BC2B23C2854D368A4EF
:1007300072C86696E0D1D87FF8D1262BF7ADBA55AE
:10074000CA15B932C3E588978E5CFB92258BBFA290
:1007500045557AA76F8B575BCF0ECB1DFB20827759
:10076000A88CCC16CE1DFADECC0B62FECCE1B7F025
:10077000C381647340A0C24D8911753355338DE830
:100780004AFDEA6E300BD7312CDE47E3BFF8554205
:10079000E27F59E517EF99346991B1238E20872DB7
:1007A000A8FED58AF3843AF037E4090054EE67498D
:1007B00093E48170E3904DEFFE41B7997BC183BA1A
:1007C00062126F7DDE6BAFDA16F95551EEA60C2B77
:1007D00002A3FD8DFB3017E46FDF3671C4CA872595
:1007E00048B047ECEAB4BFA54D9B9F0293C4E3E435
:1007F000E8422D6881150AEB845BD6A874FB7D1D49
:10080000CB2CDA462A7662CEBC5C9E8BE7CFBE78D4
:10081000F57CEBB33A9CAA6FCC72D159F21123D676
:100820003F48D1B7CEB0BFCBEA80DE57D45E972F1A
:1008300075D1508E802C6679BF724BBD8A816CD386
:10084000E101DCD21526C536DA2C1AC02794EDB7A3
:100850009B850B5E8097C5EC4FEC885D5007354754
:10086000DC0B3B3DDD60AFA85D813824255D5C1568
:10087000D1DEB3ABEC0569EF83ED5754B864641176
:10088000163269DA9F2D7F36BB445A34E87FBF03A6
:10089000EB007F59682279CF736C2C29A7A15F38B0
:1008A000A11DF02053E01A6314587110AA080C3EE1
:1008B000161A6022827FBAA443A0D0AC1BD56B6409
:1008C000B51493319E5350D05766EE5A4FFB032A0E
:1008D000695876F183F74EBA8C4206605D6DCE6042
:1008E00088AEA4C3F103A54B98A1FF67E1ACA2B801
:1008F00062D76FA031B4D277AF211006C69AFF1D20
:1009000009170E5FF1AA54344B458A8763A6DCF9B8
:10091000243067C6B2D6613369EE50615728E77E4E
:10092000EEEC3A5A734EA88DE418EAEC4164C8E242
:10093000E866B62DB6FB6A6C16B3DD4643B97300A4
:100940006A71ED4E9D251AC33C4A9515993581145F
:1009500002D6989BECD8233B8429AF0C9983A69AA6
:10096000344FFAE8D03C4BD0FBB668B89E8FCDF739
:10097000602D7A22E57DAB651B95A7A87FB67747EA
:100980007B5F8B1272D0D491EFDE19503CA78BC4E1
:10099000A9B323CB76E681F0C1048FA3B8545B974B
:1009A000AC19FF3F55272FE01D429B57FC4B4E0FC4
:1009B000CE98A9435703BDE7C894DF6E367332B4AF
:1009C000EF2E857A6EFC6C188275359007F3E49FE4
:1009D0003EDC68F3B5F31980920699A2E86FFF2E0A
:1009E0007FAE42A45FFBD40E812BC304FF2BB374F4
:1009F0004E365B9C1500C6472BE88B3DF19C039A55
:100A0000587F9B9CBF854979352E567B41143947C9
:100A10008326AA078998111B86E7737AD87D7861A7
:100A200053E979F5368D449284F91350583BA46A02
:100A30003665498E3C0EF16FD284C47E8E3F39AE4E
:100A40007C84F163378E3CCC3E448145F14BB9ED5B
:100A50006B365DBB20601A0FA3AA55773AA9AE3753
:100A60004DBAB8866BBC0850F6CCA4BD1D4072A52B
:100A700086FAE210AE3D584B97F34374A99EEB21E2
:100A8000B701A4869397EE2F4F3B86A1416F412675
:100A900090785C7F30384B3FAAECED5C6F0EAD4335
:100AA00087FD9335E601EF412690999EFB195BADDA
:100AB000D2918AE046AF65FA4F84C1A12DCF458B14
:100AC000D38550557CF96788D44EE9D76B6154A122
:100AD000A4A6A2C2BF309C409F5FD7692B24825E30
:100AE000D9D6A712541AF7559F7650A99584E66B6C
:100AF0006DB59654D6CDB3A19B46A7944DC494B47E
:100B000098E3E1E234D533160754CDB77753DB4F82
:100B10004D469DE9D49C8A36B6B838266C0EFF9CAB
:100B20001B438B80CCB93DDAC7F18AF26DB8D7741C
:100B30002F7E1EB7D34AB4ACFC79486CBC96B694F1
:100B400046572DB0A3FC1EB95260852D41D04301FC
:100B50001E1CD57DFCF3960DC7CB2A299A93DD8800
:100B60002D375DAAFB4968A09C50867F685657F9CF
:100B7000791839D4E001843361CAA5D2D6E4C98A90
:100B80004A23444EBCF0DC24A1A0C4E2073C10C4BC
:100B9000B5254B6563F480E7CF61B1718221872C65
:100BA000F59100320CECA9B59A7485E3368F764F37
:100BB0009C6DCEBCAD0A4BED7604CBC3B9339E0120
:100BC0009396697DC5A245799B045C8409ED8843B1
:100BD000C7AB931426A140B5CE4EBF2A42853E2C0A
:100BE0003B54E8121F0E9759B22789FAF2DF8E683C
:100BF00059DC06BCB6850D0622ECB1CBE504E63D1A
:100C0000B3B04173083F3C588663EB50EE1D2C3760
:100C100074A9D318A3476E9354AD0A5DB82A555DE5
:100C200078F6EEBE8E3C7669B940C234EC2AB9ED56
:100C30007E20E48D0038C7E68F44A886CEEB2AE9F3
:100C400090F14CDF32FB731B6D921E95FEB4DB6599
:100C5000DF4D23548948BF4A2E70D6D762B433295A
:100C6000B13A334C236DA676A5216348E6905DED3D
:100C700090950B7A84BEB80D5E630C62264C145AB4
:100C8000B3AC23A474A76F333005600142A028B72A
:100C9000EE1938F164808243E141271F1F90547A96
:100CA000D5232ED13DCB28BA587FDC7C9124E9286E
:100CB00051836EC5562142EDA05622A140806BA8FB
:100CC000F794CA136B0C39D9FDE9F36FA69EFC703B
:100CD0008AB3BC593C1E1D6CF97CAFF9887195EB49
:100CE0005700BD9F8C4FE12483C522EAFDD30CE25F
:100CF00017187C6A4CDE77B4539B4C81CD2360AAD5
:100D00000E25739C02793230DF74DF7519F4A51457
:100D10005CF77AA8A591847C6003063BCD50B6278A
:100D20009CFEB1DDCCD3B05924B2CAE21C81229D15
:100D3000078F8EB9BE4EFAFC3965BABF9D12375E79
:100D4000977EF389F55DF5E3098C62B5209D0C5320
:100D50008A681BD28F75175DD4E5DA756219146A3B
:100D6000262DEBF8AF37F06CA455B1BCE233C09A36
:100D7000CAB011494F689B3B6B3CCC13F6C78561E9
:100D80006842AEBBDDCD4516291DEADBC803943CA5
:100D9000EE4F8211C3EC28BD970599DED7BB5E22CA
:100DA0001FD4EB64D992D985B76A056AE42441F16E
:100DB000CDF0D83FF89E0ECD0B7A706B5A750A6A4B
:100DC0003388EC17750870102F24CFC4E9420061F6
:100DD00094CA1F3A7606FAD24881F077600345D963
:100DE00061F4A46F3DD930C3046B542AB7EC3BF4D3
:100DF0004BF5685226CEFF5D1991A0A3A5A9B1E0DD
:100E000023C40A774DF95120A3A5A9B1C100828658
:100E10008E7F5D1991A0A3C4EB540B756852078CAB
:100E20009A978D79706246EF5C1B95897141E1213B
:100E3000A1A1A1C002674C1AB6CFFD785324ABB56F
:100E4000C9F16023A5C812876D5813858892876DF4
:100E50005832C70C9A97ACDA36EE5E3EDF1DB8F218
:100E6000662FBDF87247ED5813858892878C7B55A5
:100E70000990A2C6EF3DF85324ABD42AB7EC5A36FA
:100E8000EE5E3EDF3CFA764FFD5930E246EF3DF82C
:100E900053056931C10082868E7F5D19B0E227CC8F
:100EA000FB744B148B948B756833C50892878C9AAE
:100EB000B6CF1CBAD70D98B2E62FDC1B95897160AE
:100EC00023C40A968F9CBAF66E3FFC5B15A8D22607
:100ED000AFBDF872662FDC1BB4CB148B94AAB7CDD0
:100EE000F951018082866F3DD930E227CCFB744BEB
:100EF00014AAB7CDF97043046B35C9F16023A5C8B6
:100F0000F3450892876D5832E62FBDF872664E1E83
:100F1000BEFE7E7E7E5F1D9991A0A3C40A774D1808
:100F200093A4ABD40B754910A2C6EF3DF85324AB84
:100F3000B5E833E44A16AEDE1FBCDB15A8B3C5081E
:100F40007345E931C1E121A1A1A1C002866F5C3ADC
:100F5000D70D9893A4CA16AEDE1F9D99B0E246EF56
:100F60003DF872470C9AB6CFFD5911A0A3A5C8F35E
:100F7000450892876D39F043048A96AEDE3EDF1D48
:100F80009991A0C2066F3DF872470C9A978D98937D
:100F900085887345E931E023A5A9D003848A96AEFC
:100FA000DE1FBCDB15A8D226CEFF5D1991818082A1
:100FB000672DD813A4ABD40B94AAB7CDF95120A3B5
:100FC000A5C8F345E95022C6EF5C3AD70D98938542
:100FD0008873644AF74DF95120A3C40A96AEDE3EE9
:100FE000FE7E7E7E5F3CFA764FFD7872662FBDD91D
:100FF00030C3E54812878C7B5528D2078C9A97AC72
:10100000DA178D795120A3C4EB540B948B94AAD694
:101010002EBFFC5B15A8D226AFDC1BB4EA37EC3B35
:10102000F46A37CD1893856931C1E140E325C812D0
:10103000878C9AB6CFFD5911A0C2068E7F5D38F21B
:10104000470C7B746A37EC5A36EE3FFC7A764F1CBD
:101050009B95897141006344EB542AD60F9CBAD703
:101060000D9893856931C10082868E9EBEDF3CFA61
:10107000572CDA36EE3FFC5B158971410082868E73
:101080007F5D38F247ED5813A4CAF74DF95101803E
:101090006344EB542AD62EBFDD1991A0A3A5A9B1B4
:1010A000E042068E7F5D1991A0A3C40A968F7D78D9
:1010B00072470C7B746A562EDE1FBCFA570D7951AD
:1010C000016121A1C0E325A9B1C1E14002674C1A29
:1010D000978D9893A4ABD42AD60F9C9BB4CB14AA1B
:1010E000B7CDF95120A3C4EB35C9F16042068E7F1C
:1010F0007C7A766E3FFC7A766E5E3EFE7E5F3CDBEF
:1011000015897141E121C0E344EB542AB7CDF97050
:101110006227ADD832C70C7B744B14AAB7EC3BD511
:1011200028D2076D39D120C2E74C1A978D98B2C7E3
:101130000C5928F39B4B4C3A206B633A2025752CB5
:1011400020636F6C3A2025752C20726F773A20252A
:10115000752C20707265737365643A2025750A00DA
:10116000436F6E735D20583A2025642C20593A2035
:1011700025640A00507265205D20583A2025642CB1
:1011800020593A2025640A0044656C745D20643A55
:1011900020256420743A2025750A00537461727406
:1011A000696E67206D6F74696F6E2E0A004F505420
:1011B000313A2025642C204F5054323A2025640ABD
:1011C00000F400F600F500F700F80001000100014E
:1011D0000001000100010001000100010001000107
:1011E00000010001000100010001000100010001F7
:1011F00000010001000100010001000100010001E7
:1012000000010001000100010001000100010001D6
:101210000044454255473A2064697361626C6564D5
:101220002E0A0044454255473A20656E61626C655E
:10123000642E0A0000000000000000002A2B280095
:101240000000000000000000000000000000002975
:10125000000000002C1E3420212224342627252EB5
:10126000362D3738271E1F202122232425263333ED
:10127000362E37381F0405060708090A0B0C0D0E19
:101280000F101112131415161718191A1B1C1D2FE5
:101290003130232D350405060708090A0B0C0D0E05
:1012A0000F101112131415161718191A1B1C1D2FC5
:1012B0003130354C0000000000000000000000004C
:1012C00000000000000000007E0F00D4FFFFFFC7F9
:1012D000000000780A0025303862003A20002530EE
:1012E0003258000A722F63203031323334353637AA
:1012F0000A000A002530325820006B6579626F6160
:1013000072645F7265706F72743A20000A00253053
:101310003258006B6579626F6172645F7365745FE8
:101320006C65643A20005B735D004B6579626F61A8
:1013300072642073746172742E0A005B575D005BE7
:10134000535D005B525D005B445D005B435D0004E8
:101350000330000000140354007200610063006B4E
:1013600000620061006C006C000000120350006C11
:10137000006F006F007000790043006F00000004F0
:1013800003090409029400050100A03209040000C9
:10139000010301010009211101000122400007059C
:1013A0008103080001090401000203000000092173
:1013B0001101000122220007058303200001070517
:1013C00004032000010904020001030102000921B5
:1013D00011010001224D00070582030800010904E4
:1013E0000300010300000009211101000122320065
:1013F0000705850320000109040400020300000022
:1014000009211101000122220007058603200001A5
:101410000705060320000112011001000000084327
:101420005042540100010203010631FF0974A10179
:101430000975150026FF00952075088102097615AB
:101440000026FF00952075089102C00660FF096123
:10145000A1010962150026FF009520750881020987
:1014600063150026FF00952075089102C00501094B
:1014700080A101850319012AB700150126B700953F
:101480000175108100C0050C0901A1018504190135
:101490002AA002150126A002950175108100C00541
:1014A000010902A1010901A1000509190129051578
:1014B00000250195057501810295017503810105DE
:1014C00001093009311581257F95027508810609CA
:1014D000381581257F950175088106050C0A3802AB
:1014E0001581257F950175088106C0C00501090693
:1014F000A101050719E029E71500250195087501E7
:1015000081029501750881010507190029FF150061
:1015100026FF009506750881000508190129059523
:101520000575019102950175039101C011241FBE3B
:10153000CFEFDAE0DEBFCDBF04B603FE27C0809157
:10154000530390915403A0915503B09156038730F3
:10155000904BA740B04BD1F4109253031092540318
:10156000109255031092560314BE84B7877F84BF30
:101570000FB6F894A8958091600088618093600010
:10158000109260000FBEE0E0F8E3099511E0A0E0E2
:10159000B1E0EAE4F6E602C005900D92A03AB10788
:1015A000D9F723E0A0EAB1E001C01D92A335B2074C
:1015B000E1F70E94C42C0C9423330C940000FF9399
:1015C000EF93E091A001F091A101309709F0099506
:1015D000EF91FF910895FC018591803011F0EFDFCC
:1015E000FBCF0895FF27E0E230E247FF0CC04195B2
:1015F00097FF09C0EDE26095709580959095611D0B
:10160000711D811D911D27FF02C0219530E350E21D
:10161000AA27660F771F881F991FAA1FA41710F00B
:10162000A41B63955A95A9F7AA3008F0A95FA05D9D
:10163000AF93F395611571058105910541F7ED3281
:1016400011F4EF93F395F21718F43F93F395FBCF52
:101650008F91B5DFFA95E1F70895E991F9918591B8
:10166000803021F0853219F0AADFF9CF089520E00B
:10167000E89455915532C1F3503311F46894559163
:101680005A3348F4505390F3220F022E220F220FA8
:10169000200D250FF4CF0EF42195899199915336A1
:1016A00019F3533729F1533559F1BC01882799278C
:1016B000E8945C3621F48991999168945591543657
:1016C00039F446EF7EF077FF0DC08FEF9FEF0AC031
:1016D00055374AE039F0583540E121F0523642E0C2
:1016E00009F00895FF93EF937DDFEF91FF91B7CF5E
:1016F000FF93EF93FC0181918030B9F360DFFBCF62
:10170000FF93EF9368DFF1CFDF93CF93CDB7DEB7D1
:101710002596A3DFCF91DF9108959091140290FF59
:1017200045C080FD02C070E301C071E381FD02C0CD
:1017300060E301C061E382FD02C050E301C051E3F8
:1017400083FD02C040E301C041E384FD02C030E3F9
:1017500001C031E385FD02C020E301C021E386FD25
:1017600002C090E301C091E3881F8827881F805D35
:101770001F927F931F926F931F925F931F924F93BD
:101780001F923F931F922F931F929F931F928F93AD
:1017900085E291E09F938F930E94840B8DB79EB753
:1017A00042960FB6F8949EBF0FBE8DBF089522E0FB
:1017B00030E043E060E080E30E94D81C92E09A951C
:1017C000F1F700C0089582E08A95F1F700C00C940B
:1017D000811DCF93DF93C82FD62F803511F0109243
:1017E000A2010E94D70B8C2F80680E94511D8D2F63
:1017F0000E94511DEC0185E38A95F1F7000087EC0A
:1018000090E00197F1F700C000000E94811DCE0119
:10181000DF91CF910895CF93C82F0E94D70B8C2FC3
:101820008F770E94511D0E94691DC82F82E08A9502
:10183000F1F700C082E38A95F1F700C00E94811D94
:101840008C2FCF910895CF93DF93EC010E94D70B9B
:10185000CE0164E670E00E94A632615071096837DB
:10186000710510F067E770E08FE00E94E90BDF91EF
:10187000CF910C94811DCF93DF9360E080E10E94B3
:10188000E90B64E181E10E94E90B6DE183E10E94D3
:10189000E90B8FE19EE40197F1F700C0000068E1D9
:1018A00083E10E94E90B0E94D70B82EE0E94511D3A
:1018B00098E29A95F1F7C7E3D1E081E1C533D80703
:1018C00049F0FE0184910E94511DF8E2FA95F1F76A
:1018D0002196F3CFEFE8F1E03197F1F700C0000077
:1018E0008AE20E940B0C60E080E10E94E90B0E94FA
:1018F000811D8FE19EE40197F1F700C00000DF91A8
:10190000CF910895CF93DF9380E00E940B0CD82FE6
:101910008FE30E940B0CC82F8AE20E940B0CD2347A
:1019200041F4CD3B31F491E0843009F090E0892F0F
:1019300001C080E08170DF91CF9108950E94D01C9A
:101940001092A2010E94811D0E94D70B0E94811D4E
:1019500066EB8BE30E94E90B2FEF82E597E02150C5
:1019600080409040E1F700C000000E94D70B2AE6BB
:101970002A95F1F700C00E94E30B8AE68A95F1F7F9
:1019800000C06AE58AE30E94E90B9FE728E381E053
:10199000915020408040E1F700C0000082E00E94AA
:1019A0000B0C83E00E940B0C84E00E940B0C85E082
:1019B0000E940B0C86E00E940B0C0E943B0C0E94C4
:1019C000E30B8FE19EE40197F1F700C0000080E493
:1019D00096E00E94230C8FEC97E00197F1F700C08E
:1019E00000000C94820C9F92AF92BF92CF92DF9234
:1019F000EF92FF920F931F93CF93DF93EC018091AF
:101A0000A201811113C08091140280FF08C08CE1F3
:101A100091E09F938F930E94840B0F900F9060E052
:101A200080E50E94E90B81E08093A2010E94D70B20
:101A300080E50E94511D8DE58A95F1F700000E9416
:101A4000691DF82E80E00E94511D0E94691D6C01E5
:101A50000E94691DB82E0E94691D8C010E94691D9B
:101A6000E82E0E94811D8F2D0E948D0B8C2D0E94CF
:101A70008D0B8B2D0E948D0B802F0E948D0B8E2D38
:101A80000E948D0B8091140280FF08C08AE191E0D2
:101A90009F938F930E94840B0F900F909F2C991C03
:101AA0009924991CAA24A394F3FCA12C8B2D0B2C14
:101AB000000C990B982F8827C82AD92AD194C19451
:101AC000D1088E2D0E2C000C990B982F8827082BEF
:101AD000192B1195019511090E94811D8F2D877079
:101AE00011F01092A201F8829982AA82DC82CB8244
:101AF000BD821F830E83E886CE01DF91CF911F91B7
:101B00000F91FF90EF90DF90CF90BF90AF909F909C
:101B100008951092EB02109263021092A7028FEFC9
:101B200093E09093A9028093A8021092EE02109283
:101B3000ED021092AA021092320310923903109211
:101B400038031092360310923503109264021092FB
:101B5000A6029093340380933303109224021092D0
:101B600023021092EF02109265021092F30210927B
:101B7000F2021092AC021092AB021092EC021092A0
:101B800037031092F1021092F00210926702109245
:101B900066020895FC01208131812E3131052CF43B
:101BA0002F5F3F4F3183208308951182108281E09F
:101BB000FB01808308952F923F924F925F926F9224
:101BC0007F928F929F92AF92BF92CF92DF92EF92CD
:101BD000FF920F931F93CF93DF9300D0CDB7DEB763
:101BE000FC013B012A013A832983DB018D919C9101
:101BF0001197E817F90714F4ED93FC93D2018D9136
:101C00009C9111978E179F0714F4ED93FC93D201CA
:101C10002D903C90D3012D913C91C101821B930BDF
:101C20008A3091050CF451C063E070E00E94BA3232
:101C3000620F731FE617F707ACF4F8018081882361
:101C400069F0D401ED91FC91EE0FFF1FEC0DFD1D2D
:101C500031822082698D7A8DC40118C081E0E981CA
:101C6000FA8132C06E177F0784F5A981BA818C9101
:101C7000882341F1D501ED91FC91EE0FFF1FEE0D90
:101C8000FF1D318320836F89788DC5010E94CA0DA5
:101C9000F30120813181D2018D919C91821B930BA4
:101CA00097FD019695958795820F931FF301918378
:101CB0008083D2018D939C93E981FA811082D801AF
:101CC0001C9203C081E0F8018083A98DBA8D8C91AC
:101CD000882381F0F6019601225C3F4F80E090E07E
:101CE00041915191840F951F2E173F07C9F76FE15E
:101CF00070E015C0F401608171816115710599F082
:101D0000F60120E030E080E090E0261737073CF451
:101D100041915191840F951F2F5F3F4FF6CF0E9445
:101D2000BA329B0103C0D2012D913C91EF89F88D0D
:101D30008081882381F0F701A701425C5F4F80E03A
:101D400090E061917191860F971F4E175F07C9F759
:101D50006FE170E015C0D5016D917C916115710541
:101D600099F0F70140E050E080E090E04617570717
:101D70003CF4A191B1918A0F9B1F4F5F5F4FF6CF4B
:101D80000E94BA32FB0103C0D301ED91FC91C9015D
:101D90008E1B9F0B63E070E00E94BA32CB018E0F66
:101DA0009F1F0F900F90DF91CF911F910F91FF9088
:101DB000EF90DF90CF90BF90AF909F908F907F90EB
:101DC0006F905F904F903F902F9008958F929F92C9
:101DD000AF92BF92CF92DF92EF92FF920F931F9339
:101DE00026EA32E03F932F9324E632E03F932F938D
:101DF00025E3822E23E0922E38E3A32E33E0B32E88
:101E00004DEAC42E42E0D42E54EFE52E52E0F52EDA
:101E100002E313E02AEA32E04DEE52E068EA72E0B3
:101E20000E94DB0D9093F1028093F0020F900F90CF
:101E30000F900F901F910F91FF90EF90DF90CF9038
:101E4000BF90AF909F908F9008958F929F92AF9286
:101E5000BF92CF92DF92EF92FF920F931F9327E3EF
:101E600033E03F932F932CEE32E03F932F932BEAF6
:101E7000822E22E0922E32EFA32E32E0B32E48E6DD
:101E8000C42E42E0D42E55E2E52E52E0F52E05E6B2
:101E900012E02FEE32E043E252E063E373E00E948F
:101EA000DB0D90936702809366020F900F900F9066
:101EB0000F901F910F91FF90EF90DF90CF90BF9008
:101EC000AF909F908F9008950F931F93CF93DF93C0
:101ED0008C01EB0180916402882321F08091A6029D
:101EE000811103C0C8010E94E60E8091EC02882394
:101EF00021F080913703811103C0CE010E94250F8C
:101F00004091F0025091F102809166029091670237
:101F10002091EB02211121C0041715077CF4C8178A
:101F2000D9070CF469C083E08093EB028091A7028B
:101F3000882309F461C01092A70238C0C817D907D6
:101F40000CF05AC081E08093EB02809163028823F9
:101F500009F452C01092630238C02130B1F4041762
:101F600015073CF0C817D9070CF446C01092EB02D5
:101F700007C0C817D9070CF03FC082E08093EB027E
:101F80002093A7021092630237C0223009F504178C
:101F900015077CF0C817D9077CF581E08093EB0228
:101FA00080916302882341F11092630281E090E006
:101FB00025C0C817D90704F183E08093EB02809114
:101FC000A7028823C9F01092A7028FEF9FEF16C0D7
:101FD0000417150734F0C817D90774F01092EB02F4
:101FE00006C0C817D90744F482E08093EB0281E071
:101FF000809363021092A70280E090E0DF91CF917E
:102000001F910F910895FC01648343830895EF921B
:10201000FF920F931F93CF93DF93EC018091A40164
:102020009091A5010E94DA298436910508F44CC0EC
:102030008091A6019091A7010E94DA29059708F4E2
:1020400043C08091AA0181113FC00E94C229909390
:10205000A7018093A60180E00E94AD1C8C0184E062
:102060000E94AD1C7C018091A3018823A1F0809186
:10207000140280FF10C0FF92EF921F930F938DEA1E
:1020800091E19F938F930E94840B0F900F900F907C
:102090000F900F900F90B701C8010E94640F882322
:1020A00099F04B81042E000C550B480F511D6C818B
:1020B000062E000C770BCE01DF91CF911F910F916F
:1020C000FF90EF900C940310DF91CF911F910F912F
:1020D000FF90EF900895FC01618342830895AF92D1
:1020E000BF92CF92DF92EF92FF920F931F93CF9305
:1020F000DF93CDB7DEB729970FB6F894DEBF0FBEDA
:10210000CDBF6C01CE0101960E94F30C8B81882318
:1021100009F4AAC08A81882309F4A6C00C811D8114
:10212000AF80B8848091A8019091A901892BA1F476
:102130008091140283FF0AC080FF08C08BE991E1FF
:102140009F938F930E94840B0F900F900E94C2293F
:102150009093A9018093A8018091140283FF24C069
:1021600080FF22C08091A9018F938091A8018F9355
:10217000980117FF03C0319521953109C501B7FEBC
:1021800003C0919581959109820F931F9F938F931F
:1021900088E891E19F938F930E94840B0F900F909A
:1021A0000F900F900F900F908091140283FF12C038
:1021B00080FF10C0BF92AF921F930F9384E791E10D
:1021C0009F938F930E94840B0F900F900F900F900E
:1021D0000F900F907801003811051CF09FE7E92E51
:1021E000F12C81E8E8168FEFF80624F481E8E82E58
:1021F000FF24FA9485010038110514F00FE710E070
:1022000001388FEF180714F401E81FEF80911402D2
:1022100083FF12C080FF10C01F930F93FF92EF92B5
:1022200080E691E19F938F930E94840B0F900F9013
:102230000F900F900F900F9044275527401B510B84
:10224000B701C60129960FB6F894DEBF0FBECDBF09
:10225000DF91CF911F910F91FF90EF90DF90CF9082
:10226000BF90AF900C946B1029960FB6F894DEBF18
:102270000FBECDBFDF91CF911F910F91FF90EF90D7
:10228000DF90CF90BF90AF900895DF92EF92FF92D2
:102290000F931F93CF93DF9300D000D01F92CDB741
:1022A000DEB78C017B01FB0182811F928F938181BC
:1022B0001F928F9380811F928F931F930F9385E3BB
:1022C00091E19F938F930E94840B0FB6F894DEBF29
:1022D0000FBECDBFF7018081813069F4818181110A
:1022E0000AC00E94C2299093A5018093A401F7011E
:1022F00082818093AA01B701C8010E94D212D82E10
:10230000882309F448C00932FDE51F0719F5F701D4
:1023100082818823F9F080913A0390E0019663E08E
:1023200070E00E94A63280933A0360913A03709164
:102330003B0380913C0390913D030E948628E091ED
:102340003A03F0E0EE0FFF1FE050FF4F80819181D4
:102350000E94230C045F110905301105E0F40E946E
:1023600072173A834B835C836D83F701828141E06E
:1023700050E001C0440F0A95EAF7882311F0422B80
:1023800002C0409542235A816B817C818D810E94DD
:1023900092170E9467178D2D0F900F900F900F903E
:1023A0000F90DF91CF911F910F91FF90EF90DF90F1
:1023B00008950F931F93CF93DF93CDB7DEB72B977D
:1023C0000FB6F894DEBF0FBECDBF80988898849872
:1023D0008C988BE0E5E1F1E0DE01119601900D9221
:1023E0008A95E1F7FE0131969E01245F3F4F41E05F
:1023F00050E08191A82FA295AF70B0E091966C91BA
:1024000091978F708A0102C0000F111F8A95E2F721
:10241000C801962F982B91969C93919792969C9198
:1024200092978095892392968C932E173F0709F7F0
:10243000879A8091140280FF02C08F9A01C08F9802
:102440002B960FB6F894DEBF0FBECDBFDF91CF91B4
:102450001F910F910C944A1E0E949E0C0C94890DA2
:10246000EF92FF920F931F93CF93DF93CDB7DEB719
:102470002A970FB6F894DEBF0FBECDBF8D834111F2
:1024800016C0E11014C0511112C0F11010C061113A
:102490000EC001110CC08D81811109C0211107C02E
:1024A000711105C081E0111103C080E001C081E01D
:1024B00081702A960FB6F894DEBF0FBECDBFDF91B4
:1024C000CF911F910F91FF90EF900895EF92FF929F
:1024D0000F931F93CF93DF93CDB7DEB72A970FB635
:1024E000F894DEBF0FBECDBF0E9472172E833F83CC
:1024F000488759876A87CE0106960E940710CE0149
:1025000006960E946F104E815F81688579858A8565
:102510000E9492170E94721779018A01262F4E811C
:102520005F81688579858A850E94301281110E94B9
:1025300067172A960FB6F894DEBF0FBECDBFDF91A6
:10254000CF911F910F91FF90EF90089581E08093BC
:102550003A0360913A0370913B0380913C03909160
:102560003D030C9486280E94822860933A0370935E
:102570003B0380933C0390933D03643010F00E9432
:10258000A6120C94C216E0913A03F0E0EE0FFF1F82
:10259000E050FF4F808191810E94230C0C94481ED3
:1025A00081E0089581E0089508950C94D4121F935A
:1025B000CF93DF9300D000D01F92CDB7DEB7498311
:1025C0005A836B833091C10189819A81311114C082
:1025D000662359F0222349F00E940F27182F682FF5
:1025E00089819A810E94B62603C00E94E226182F94
:1025F00069817A81812F04C00E940F2769817A81C5
:102600000F900F900F900F900F90DF91CF911F912F
:102610000C94A519FC01262F4081518162817381A0
:1026200084810C94D712CF93DF93EC0160E00E9479
:102630000A13BE01DF91CF910C94D512FF920F9334
:102640001F93CF93DF93E82FF0E0EC5CFD4EF49006
:10265000C82FC695C695C695D0E0FE01EC53FD4E39
:102660000491877010E0082E02C0159507950A9412
:10267000E2F701701127FE01EC54FD4EC491D0E049
:1026800002C0D595C7958A95E2F7C170DD2701157F
:10269000110519F081EE0E94371F209719F086EE80
:1026A0000E94371F8F2D0E94B11FCD2B19F086EE8F
:1026B0000E94851F012B41F081EEDF91CF911F9188
:1026C0000F91FF900C94851FDF91CF911F910F9177
:1026D000FF900895EF92FF920F931F93CF93DF9394
:1026E000EC01162F0AE08881882309F455C0813057
:1026F00009F043C08981813041F47E0182E0E80E17
:10270000F11C8A810E94B11F09C0823049F47E0108
:10271000E2E0EE0EF11C8A810E94371FE7012FC014
:10272000833041F47E01F2E0EF0EF11C8A810E94B9
:10273000851FF4CF843011F0219621C02A81229682
:1027400080E090E030E0205331092A30310558F420
:10275000089FA001099F500D1124C901840F951FE6
:1027600021962881EFCF009751F0EFECF7E03197F9
:10277000F1F700C000000197F6CF0E941E132196CA
:10278000812F882309F4AFCFEFECF7E03197F1F711
:1027900000C000008150F5CFDF91CF911F910F91C4
:1027A000FF90EF90089560E00C946A138F929F92CF
:1027B000AF92BF92CF92DF92EF92FF920F931F934F
:1027C0006B017C0181E090E0A0E0B0E04C015D0194
:1027D00004C0880C991CAA1CBB1C4A95D2F7AC01FA
:1027E000BD0104C0440F551F661F771F2A95D2F7FD
:1027F000482959296A297B2904C0880F991FAA1FD3
:10280000BB1F0A95D2F78A019B010C211D212E21A5
:102810003F21401751076207730739F4BC01CD010E
:102820006C297D298E299F290AC080959095A095B5
:10283000B095BC01CD016C217D218E219F211F917E
:102840000F91FF90EF90DF90CF90BF90AF909F904F
:102850008F9008950F93382F262F6091FF0170916C
:1028600000028091010290910202042F432F0E94E6
:10287000D6130F910C94F2250E94352A0E945128FC
:10288000811102C00E94EA280C94B3120C94C01665
:1028900008950E943C220E9448142FE78AE196E0A6
:1028A000215080409040E1F700C000000C940F2AB6
:1028B0000F931F93CF93DF93EC0161E00E940A1303
:1028C0008C01BE010E940C18882309F449C0BE0186
:1028D000C8010E944511882309F442C0BE01C80105
:1028E0000E94FF1A8823E1F1BE01C8010E94511B1A
:1028F0008823B1F1BE01C8010E947C1C882381F1AC
:102900008A81882331F101308CE5180751F00F3DA1
:102910008CE51807D9F001151C45D9F40E9449141B
:102920001FC080911402C82FC095C170C0FB80F9F0
:1029300080931402CC2329F083E292E10E94EB0AF7
:102940000FC081E192E10E94EB0A0BC00E94EA28CD
:1029500007C0CE01DF91CF911F910F910C94D0123F
:10296000C0E08C2FDF91CF911F910F9108950895B2
:102970000C94B71481E008950C94BA14CF93C82F27
:102980000E94B8148C2F0E94BC14CF910895CF934D
:10299000DF930E94A5190E94B815EC01811592459C
:1029A000F0F5C11581E5D80708F0A9C0C83ED105EA
:1029B00028F5C03ED10508F0D7C0C83AD10578F453
:1029C000C53AD10508F074C0C130D10509F4CCC0B6
:1029D00008F4C8C0C430D10508F0C6C0C3C0CF3B9E
:1029E000D10508F0BFC0C85AD0E0CC0FDD1FC05ED3
:1029F000DE4F0990D881C02DD464B6C0C11590E5D2
:102A0000D90708F060C0C11520E4D20708F058C00B
:102A1000CE019A9581159F4108F4A6C0A3C0C115A7
:102A200086E5D80718F5C11595E5D90708F080C0E7
:102A3000C11524E5D20708F076C09E012370332724
:102A40008C2F86958695C115D34508F05DC0C1E0F1
:102A5000D0E002C0CC0FDD1F2A95E2F720E2829F72
:102A6000C0011124C82BD92BDC687EC0C1152AE512
:102A7000D20778F4C11589E5D80708F063C0C115FD
:102A800098E5D90708F46EC0DC2FCC27C06FD06A58
:102A90006BC0CE0190568115904208F063C08D2F17
:102AA0008F710E944C16DD27D0628F71D82B5CC0CD
:102AB000C55AD0E0C25BDE4FC881D0E0D06454C0BC
:102AC000DF70D06A51C0CE0174E0969587957A95F3
:102AD000E1F783709C2F937021E030E002C0220F59
:102AE000331F9A95E2F73C68382BCF70C695C69590
:102AF00080E2C89FE0011124C22BD32B35C0DC2F0C
:102B0000CC27C16FD06A30C0C1E0D0E002C0CC0F8A
:102B1000DD1F2A95E2F720E2829FC0011124C82B15
:102B2000D92BDA6821C0DC2FCC27C46FD06A1CC037
:102B30008C2F0E944C168F71C82FD0E0DC2FCC2731
:102B4000D06212C08C2F8F700E944C1694E0D695E4
:102B5000C7959A95E1F7CF70D0E0DC2FCC27D069EC
:102B6000C82B02C0C0E0D0E0CE01DF91CF91089524
:102B70008238910569F1B0F48133910509F46DC093
:102B800048F48932910509F463C08A32910509F449
:102B900069C008958533910509F455C089339105BD
:102BA000B9F00895833E910569F138F4803E9105AE
:102BB000B1F0823E910509F10895863E9105A9F193
:102BC000873E9105B9F1843E910509F064C023C0A8
:102BD0002091440320FD4FC021FD4DC008958091F8
:102BE000440380FD44C08091450380FF44C0809130
:102BF000440384FD42C083EE4DC08091440382FFB4
:102C000038C0F5CF8091440382FD33C080914503E5
:102C100080FD31C0ECCF8091450381FF32C08091AF
:102C2000440384FD2AC087EE35C08091440383FFAE
:102C300026C0F5CF8091440383FD21C080914503D8
:102C400081FD1FC0ECCF8091440385FD1CC01DC0D9
:102C50008091440385FD19C016C08091440386FD10
:102C600016C017C08091440386FD13C010C089E3CD
:102C700011C082EE0FC080EE0DC080E00BC086EE6A
:102C800009C084EE07C089E205C085E303C08AE27B
:102C900001C081E390E008959091440392FF0DC03C
:102CA000282F2871283019F4877F846006C0282FC8
:102CB0002471243011F48B7F886093FF0DC0282F7E
:102CC0002871283119F4877E846106C0282F247169
:102CD000243111F48B7E88612091450320FF0DC0C3
:102CE000382F3871383019F4877F816006C0382F4B
:102CF0003171313011F48E7F886021FF0DC0282F93
:102D00002871283119F4877E816106C0282F21712E
:102D1000213111F48E7E886194FD877E0895E82F1D
:102D2000F0E0E15CFC4F8081089583EE92E10E9427
:102D3000EB0A1F921F928EED92E19F938F930E9458
:102D4000840B8BED92E10E94EB0A80913F030E947D
:102D500039281F928F9386ED92E19F938F930E9463
:102D6000840B8DB79EB708960FB6F8949EBF0FBE22
:102D70008DBF84ED92E10C94EB0A08950C94BD167E
:102D80000C94BE160C94BD16CF93DF93A1E5B1E071
:102D900066E571E041E050E08D918F3F71F46A1774
:102DA0007B07D1F710923E0310923F0381E00E940F
:102DB0003017DF91CF910C943C14E82FE295EF701F
:102DC000F0E021A18F70EA0102C0CC0FDD1F8A95CF
:102DD000E2F7CE019C2F9095922391A392A1892B8B
:102DE00082A3DDCFCF93A1E5B1E040E050E030E039
:102DF00061E070E02D912F3FC1F0E22FE295EF707E
:102E0000F0E080A190E02F7002C0959587952A95FB
:102E1000E2F780FD07C0CB01042E01C0880F0A94A1
:102E2000EAF702C080E090E0382B4F5F5F4F4530FB
:102E3000510501F780913E03831721F030933E0343
:102E4000C1E001C0C0E02C2F41E06FE373E08EE3EE
:102E500093E00E9431170E9446148C2FCF91089561
:102E60000895FF920F931F93CF93DF938C01F62E5B
:102E7000D72FC42F222349F081E08093AD010E9417
:102E8000C2299093AC018093AB018091AD0188235E
:102E9000C1F08091AB019091AC010E94DA290697B4
:102EA00080F0EF2DFD2FD8014C2F50E0CD01801B7D
:102EB000910B841795071CF48D918193F7CF109295
:102EC000AD01DF91CF911F910F91FF9008958EEA90
:102ED00091E00E94031EEEEAF1E011821282138259
:102EE00014820895CF93DF9300D000D01F92CDB706
:102EF000DEB785E0EEEAF1E0DE01119601900D9279
:102F00008A95E1F729813A814B815C816D8170E07E
:102F100080E090E00F900F900F900F900F90DF9156
:102F2000CF910895CF93DF9300D000D01F92CDB7FB
:102F3000DEB749835A836B837C838D8385E0FE01F2
:102F40003196AEEAB1E001900D928A95E1F70F90CB
:102F50000F900F900F900F90DF91CF91089582E224
:102F600090E00E94DB32813281F483E290E00E94A3
:102F7000DB32823051F484E290E00E94DB3291E057
:102F8000893109F090E0892F01C080E081700895B7
:102F9000CF93C82F811102C06FEF01C061E282E2BE
:102FA00090E00E94EF32C11102C06FEF01C062E0F9
:102FB00083E290E00E94EF32C11102C06FEF01C0C6
:102FC00069E184E290E0CF910C94EF3280E00E94BE
:102FD000C8170C944B28089585E290E00E94DB32DC
:102FE000682F70E080E090E0089585E290E00C9416
:102FF000EF320E94EB170E94AF1781110CC060E006
:1030000070E0CB010E94F5170E9439190E94FF1948
:1030100081E00C94C8170895CF93FB01C281CC23A3
:10302000E9F09C0122513F452031310520F48251C5
:103030000E940F1A0CC08031FFE59F0751F481E018
:103040000E94182643E062E081E00E942A14C0E05A
:1030500018C081319F45A9F482E0F2CF8031EFE5BD
:103060009E0711F481E004C081319F4549F482E05C
:103070000E94392643E062E081E00E942A1401C0E8
:10308000C1E08C2FCF9108952FEFFC01208308958C
:103090001F93CF93DF93EC01162FE8818E2F90E0E2
:1030A000FC013197E331F10508F094C0EA5AFF4F73
:1030B0000C94CE32198289E099C08981823041F026
:1030C000833009F490C08130B1F40E94CE2902C04F
:1030D0000E94EC179A838B837C836D837DC08981EA
:1030E000823049F46A817B818C819D810E94D43237
:1030F0000E94F51771C0612FCE010E9444186CC068
:103100004B816A8189810E940B199C838D8364C0E5
:103110002C813D813227232732274B816A81898187
:103120000E94241959C00E94391956C00E94B21930
:1031300023C00E94B419998359C06B8170E08981C2
:103140009A81AE014C5F5F4F9827892798270E948C
:10315000B71942C06B8170E089819A81AE014C5FE2
:103160005F4F9827892798270E94DC1935C00E9455
:10317000FF1932C00E94F81889832EC06B8170E05D
:1031800089819A81AE014C5F5F4F982789279827E4
:103190000E94611921C06B8170E089819A81AE0122
:1031A0004C5F5F4F9827892798270E94841914C085
:1031B0000E94E61711C0CE010E94572B2FEF80E727
:1031C00092E0215080409040E1F700C000000E9452
:1031D0000F2A02C08FEF8883612FCE01DF91CF913C
:1031E0001F910C94572B80E00E948F168A83F4CF96
:1031F00088E0089550E0440F551F2AE0629F400D7B
:10320000511D11249A016AE0869F200D311D112461
:10321000C901869608950F931F93CF93DF930E9461
:10322000FA188C010E94DB32C82FD0E0DC2FCC27AB
:10323000C80101960E94DB329E01282BC901DF9153
:10324000CF911F910F9108950F931F93CF93DF9309
:10325000122F032F0E94FA18EC01602F0E94EF3208
:10326000612FCE010196DF91CF911F910F910C94A8
:10327000EF32FF920F931F93CF93DF93F12C00E077
:1032800010E0C0E0D0E0FE01E00FF11FEE0FFF1FE5
:10329000EF53FE4E259134914C2F60E08F2D0E940C
:1032A00024192196C530D10571F70B5F1F4FF39498
:1032B00088E0F812E6CFDF91CF911F910F91FF9038
:1032C0000895EF92FF920F931F93CF93DF93EA013C
:1032D0007A01E60EF71E8C01C8018696CE15DF0531
:1032E00061F00035110520F40E94DB32888301C0B3
:1032F000188221960F5F1F4FEFCFDF91CF911F9163
:103300000F91FF90EF900895EF92FF920F931F930C
:10331000CF93DF93EA017A01E60EF71E8C01C80114
:103320008696CE15DF0551F00035110518F4688139
:103330000E94EF3221960F5F1F4FF1CFDF91CF91A7
:103340001F910F91FF90EF900895462F883038F429
:10335000711105C0653018F460E00C940B1980E021
:1033600090E0089580E108958AE893E00895EF924F
:10337000FF920F931F93CF93DF93EA017A01E60E3A
:10338000F71E8C01C8018A589F4FCE15DF0569F0E2
:103390000A3823E0120720F40E94DB32888301C040
:1033A000188221960F5F1F4FEDCFDF91CF911F91B4
:1033B0000F91FF90EF900895EF92FF920F931F935C
:1033C000CF93DF93EA017A01E60EF71E8C01C80164
:1033D0008A589F4FCE15DF0559F00A3823E01207AF
:1033E00018F468810E94EF3221960F5F1F4FEFCFD4
:1033F000DF91CF911F910F91FF90EF900895CF93A0
:10340000DF93C6E7D0E060E0CE010E94EF32219664
:10341000C11584E0D807B9F7DF91CF910895DF9205
:10342000EF92FF920F931F93CF93DF9300D000D0C2
:10343000CDB7DEB7F82E8FE08F15E8F18FEF93E070
:103440000E94DB32811137C006E710E0FF2069F0EF
:10345000011584E0180779F1C8010E94DB3281115F
:1034600001C0FA940F5F1F4FF1CF19821A821B829D
:103470001C82DD24D39478018FEFE81AF80AC80182
:103480000E94DB3289831A828823A9F09FEF980F6C
:10349000933058F48A83D9820E5F1F4FC7010E9470
:1034A000DB328B83882339F07801CE0101960E94AC
:1034B000D3138701E0CF0F900F900F900F90DF9103
:1034C000CF911F910F91FF90EF90DF900895AF92F1
:1034D000BF92CF92DF92EF92FF920F931F93CF9301
:1034E000DF937C015B01C42FD22FFC0182818823F2
:1034F000F9F04093B5010E94C2299093B4018093E2
:10350000B30180E28C0F883008F06EC0C77081E094
:1035100001C0880FCA95EAF7DF91CF911F910F91F3
:10352000FF90EF90DF90CF90BF90AF900C94C41FAE
:103530008091B501481335C08091B3019091B401D9
:103540000E94DA296C01B701C5010E94F524C81652
:10355000D90638F510E21D0FCD17B9F080E28C0FB7
:10356000883040F4C77081E001C0880FCA95EAF73F
:103570000E94CB1F183058F581E09D2F977001C035
:10358000880F9A95EAF70E94C41F802F0E94B11FEE
:10359000183050F5D77081E001C0880FDA95EAF74E
:1035A0000AC080E28C0F8830F8F4C77081E001C057
:1035B000880FCA95EAF7DF91CF911F910F91FF9085
:1035C000EF90DF90CF90BF90AF900C94CB1F802FE7
:1035D000DF91CF911F910F91FF90EF90DF90CF90EF
:1035E000BF90AF900C94B11FDF91CF911F910F91BD
:1035F000FF90EF90DF90CF90BF90AF9008950F9322
:103600009C01CB01243F4CE5340731F188F4293D7E
:10361000FCE53F07D9F02A3D4CE5340779F1283D18
:103620003C45A9F506E221EE41EE68ED7CE52BC0B4
:10363000263FFCE53F07E1F0A8F0273F3C4539F580
:1036400007E225EE46EE67EF7CE51DC007E225EEBA
:1036500045EE69ED7CE517C006E221EE40EE64EF31
:103660007CE511C007E225EE44EE65EF7CE50BC07A
:1036700006E221EE42EE66EF7CE505C008E221E0BD
:1036800045EE6AED7CE50E94671A80E008C0FC0107
:103690008281882319F01092B50101C081E00F9159
:1036A0000895CF93DF93EC01FB018281882309F415
:1036B0001FC1C230FCE5DF0708F41BC1C6319CE521
:1036C000D90738F09E012B5F3C452930310508F0C1
:1036D00010C10E9464289093450380934403C03135
:1036E000ECE5DE0709F4C3C008F041C0C8308CE542
:1036F000D80709F49AC0F0F4C430ECE5DE0709F409
:1037000087C068F4C2308CE5D80709F477C0C330AD
:10371000DC4509F0E3C080914403826076C0C63086
:10372000ECE5DE0709F46EC008F07BC0809144032D
:1037300088606BC0CC308CE5D80709F485C068F48C
:10374000CA30ECE5DE0709F474C008F079C00E94C5
:103750003C2280914403806858C0CE308CE5D80765
:1037600009F476C008F07FC0809144038BC0CC3F41
:10377000ECE5DE0709F44FC018F5C3318CE5D80736
:1037800009F47DC078F4C131ECE5DE0709F473C0BB
:10379000C231DC4509F0A2C00E943C228091440362
:1037A0008F7733C0C5318CE5D80709F472C008F4AF
:1037B00086C0CB3FDC4509F091C0809145033EC0F7
:1037C000C115FDE5DF0709F45FC058F4CE3F9CE565
:1037D000D90709F444C008F43FC0809145038260D2
:1037E0002DC0C230FDE5DF0709F475C008F45DC0E7
:1037F000C330DD4509F072C080E06EC080914403A3
:10380000816003C08091440380618093440366C05B
:103810008091440311C080914503826080934503E9
:103820005DC0809144038062F0CF80914403806446
:10383000ECCF8091440388608460E7CF8160EECF55
:10384000809144038E7FE1CF809144038D7FDDCF53
:1038500080914403877FD9CF8091450318C0809120
:1038600045038D7FDBCF809144038F7ECECF809147
:1038700044038F7DCACF809144038F7BC6CF809154
:103880004403877F8B7FC1CF809145038D7F8E7FDF
:10389000C5CF8091440382FB222720F991E0922733
:1038A00090FB82F990FB83F9B0CF80914503982F6C
:1038B000909591708E7F892B90FB81F9AFCF0E94FC
:1038C0003C228091440387FB222720F991E0922734
:1038D00090FB87F99ACF81E00E94EC288091440305
:1038E000909145030E9475280E943C2280E001C00F
:1038F00081E0DF91CF910895CF93DF9386319C458E
:1039000041F5EB010E949027982F8A8120910801B0
:1039100030910901882379F09A7A81E009F480E0F6
:103920008093B601911102C069E201C065E3C9014B
:103930000E9433290AC08091B601811102C069E258
:1039400001C065E3C9010E9435290E94D12780E0AA
:1039500001C081E0DF91CF91089595E890937A00BE
:10396000982F9072906890937B008F7190910601D0
:10397000892B80937C0080917A00806480937A0008
:1039800080917A0086FDFCCF8091780020917900AB
:1039900090917A009F7790937A0090E0922B08950F
:1039A000289A219A229A23982B9880E58CBD089515
:1039B000909107019F3F09F072C08F3F09F46FC0DB
:1039C000611103C01092B80103C090E29093B80156
:1039D000423041F0433051F0413069F49091B801E8
:1039E000946007C09091B801986003C09091B801AD
:1039F0009C609093B80141E050E04217530718F4DF
:103A0000440F551FFACF9091B80140315105F1F0A4
:103A100050F442305105B1F048305105E1F421E055
:103A20002093B70113C04034510591F0403851053F
:103A300039F04032510579F421E02093B70108C0F4
:103A4000936007C091E09093B70105C0916001C0F9
:103A500092609093B8012CB59091B801922B9CBDC7
:103A60009091B701992319F09DB591609DBD809308
:103A70000701E82FE295EF70F0E031A1282F2F70B9
:103A800081E090E001C0880F2A95EAF7932F982BE8
:103A900091A392A18095892382A381E0089580E07B
:103AA0000895CF93DF938EBD0E94C229EC010DB41F
:103AB00007FC0AC00E94C2298C1B9D0B843691050D
:103AC000B0F38EEF9FEF02C08EB590E0DF91CF9103
:103AD0000895CF93DF931EBC0E94C229EC010DB460
:103AE00007FC0AC00E94C2298C1B9D0B84369105DD
:103AF000B0F38EEF9FEF02C08EB590E0DF91CF91D3
:103B00000895809107018F3F19F1E82FE295EF703A
:103B1000F0E031A1282F2F7081E090E001C0880FE4
:103B20002A95EAF7932F982B91A392A1892B82A330
:103B30008FEF809307018DB58E7F8DBD9CB58091F1
:103B4000B801809589238CBD1092B8011092B701FD
:103B500008959093BE018093BD010895E091BD0149
:103B6000F091BE01309721F00190F081E02D099491
:103B700080E00895EF92FF920F931F93CF93DF930E
:103B8000E091BD01F091BE013097B1F18C0102804E
:103B9000F381E02D09958091140282FF2DC080FFF2
:103BA00004C08AEF92E10E94EB0AE80118E084EF7A
:103BB000E82E82E1F82E8091140280FF0BC08881EC
:103BC0001F928F93FF92EF920E94840B0F900F90A1
:103BD0000F900F90115021961111EDCF809114028A
:103BE00080FF0AC082EF92E1DF91CF911F910F9188
:103BF000FF90EF900C94EB0ADF91CF911F910F9102
:103C0000FF90EF900895E091BD01F091BE013097D3
:103C100021F00480F581E02D099408952091BB01E5
:103C20003091BC012817390771F09093BC01809343
:103C3000BB01E091BD01F091BE01309721F00680FB
:103C4000F781E02D099408952091B9013091BA01CE
:103C50002817390771F09093BA018093B901E09168
:103C6000BD01F091BE01309721F00084F185E02D77
:103C70000994089585B7806885BF85B7806885BF3A
:103C8000089581E008950C94411E08950C94451EFA
:103C90000C94451E0C94451E0C94451E0E943A1E21
:103CA0000E944C1E0C94D9110E94B9290E94C4167E
:103CB0000E94F9170E94492A0E942C120C94C312E8
:103CC000CF93C82F8091140282FF1EC080FF04C0D2
:103CD00083E193E10E94EB0A8091140280FF0CC003
:103CE0001F92CF938EE093E19F938F930E94840B5A
:103CF0000F900F900F900F908091140280FF04C0DE
:103D00008CE093E10E94EB0A8C2FCF910C94BE14AF
:103D1000FF920F931F93CF93DF93CDB7DEB72A9710
:103D20000FB6F894DEBF0FBECDBF0E94461E0E94A4
:103D3000451E0E94F2160E94431E882379F180E0FE
:103D40000E948F16082FF090C001F82639F180915B
:103D5000140281FD0E94951680E011E09F2D9123B1
:103D6000C9F08E831F82012381E009F480E08887F7
:103D70000E94C2298160782F9A8789874E815F814E
:103D800068858A850E94031F8091C00118271093BF
:103D9000C00114C08F5F110F853001F78FEF898349
:103DA0008A831B820E94C2298160782F9D838C8325
:103DB00049815A816B818D810E94031F0E94661286
:103DC0000E94AE1D9091BF01891789F00E94AE1D1F
:103DD0008093BF012A960FB6F894DEBF0FBECDBF09
:103DE000DF91CF911F910F91FF900C94601E2A9646
:103DF0000FB6F894DEBF0FBECDBFDF91CF911F91FC
:103E00000F91FF900895CF93DF93CDB7DEB72B9737
:103E10000FB6F894DEBF0FBECDBF4F8358876987BA
:103E20007A878B87DE01119686E0FD0111928A95D3
:103E3000E9F785E0FE01379601900D928A95E1F74A
:103E400049815A816B817C818D819E810E94F824F9
:103E50002B960FB6F894DEBF0FBECDBFDF91CF918A
:103E60000895FC01808191810E9451270895CF938C
:103E7000882309F448C0C82F8CEF8C0F813AD0F406
:103E80006C2F80910801909109010E94FD288823E0
:103E900049F06C2F80910801909109010E94352909
:103EA0000E94D1276C2F80910801909109010E94F6
:103EB00033290CC080E28C0F883058F4C77081E041
:103EC00001C0880FCA95EAF70E949327CF910C94FE
:103ED000D127EBE5EC0FE33040F4F0E0EC57FE4F78
:103EE000808190E0CF910C940E1EC85AC73158F4CF
:103EF000EC2FF0E0EE0FFF1FEA5AFE4F8081918118
:103F0000CF910C94241ECF910895882349F1682FF6
:103F10008CEF860F813A38F4809108019091090165
:103F20000E9435290CC080E2860F883050F46770FB
:103F300081E001C0880F6A95EAF70E9499270C94E6
:103F4000D1278BE5860F833020F480E090E00C943D
:103F50000E1E685A673120F480E090E00C94241E15
:103F60000895CF93C82F0E94371FC93349F42FEF0C
:103F700083EF91E0215080409040E1F700C00000C5
:103F80008C2FCF910C94851F882321F00E949327BA
:103F90000C94D1270895882321F00E9499270C942E
:103FA000D1270895CF92DF92EF92FF920F931F9344
:103FB000CF93DF937C01D62FC72FFC01058102959B
:103FC0000F70128111110E94B0270E948927882347
:103FD00099F0112389F08C2F807F803421F080E2CA
:103FE0008D0F883048F082E00E941B280E948927AC
:103FF00091E0D82ED92601C0D12CCC2EC2948FE0CE
:10400000C8228C2D90E08C30910508F0ABC1FC01EA
:10401000E759FF4F0C94CE328C2F807FCF708823CE
:1040200011F0C295C07F112399F0CC2309F486C109
:1040300080E28D0F883010F0D11104C08C2F0E94C7
:10404000932703C08C2F0E94A3270E94D12776C1FB
:104050008D2F0E94851FCC2309F484C180E28D0F2F
:10406000883010F0D11104C08C2F0E94992703C012
:104070008C2F0E94A9270E94D12774C18C2F807F8A
:10408000CF70803211F0C295C07FDD2319F0D1309E
:10409000C9F022C0112371F0002341F0013031F446
:1040A0000E94B6278C2B0E94BE275CC10E94B627B7
:1040B0008C2B1DC0002319F0013009F453C10E945C
:1040C000C72725C0112321F0063008F04BC10EC0D0
:1040D000053008F047C11BC0112361F0002331F007
:1040E000F701858180FF2AC18F7085838C2F0E9404
:1040F000C41F38C1002359F0D93309F030C1FFEF94
:1041000003EF11E0F15000401040E1F726C18C2F81
:104110000E94CB1F27C18C2F86958695837019F03E
:10412000813061F01FC1112321F08D2F9C2F9370DE
:1041300002C080E090E00E940E1E1CC1112321F0FD
:104140008D2F9C2F937002C080E090E00E94241E6F
:1041500011C18C2F837009F047C0111107C12D2F99
:10416000229526952770220F220F6D2F6F70862FB4
:1041700090E0A0E0B0E0022E04C0880F991FAA1FB3
:10418000BB1F0A94D2F7D4FF10C04FE050E060E0AC
:1041900070E004C0440F551F661F771F2A95D2F7A1
:1041A000409550956095709503C040E050E0BA018D
:1041B000C695C695C3708A019B01082B192B2A2B23
:1041C0003B2BC901B801C23049F058F4C13019F095
:1041D0000E94CC25CBC00E94BA25C8C00E94DE2513
:1041E000C5C00E94B825C2C0112319F08C2F817060
:1041F00001C08695882309F4B9C02D2F22952695F4
:104200002770220F220F6D2F6F70862F90E0A0E095
:10421000B0E0022E04C0880F991FAA1FBB1F0A948A
:10422000D2F7D4FF10C04FE050E060E070E004C06F
:10423000440F551F661F771F2A95D2F7409550955A
:104240006095709503C040E050E0BA01C695C695F0
:10425000C3708A019B01082B192B2A2B3B2BC90108
:10426000B801C23049F058F4C13019F00E949126CB
:104270007DC00E947F267AC00E94A32677C00E943C
:10428000F22574C0CF70112339F08C2F0E941826AC
:104290008D2F0E94C41F6AC08D2F0E94CB1F8C2FB0
:1042A0000E94392663C0D23F01F128F4D03F41F08B
:1042B000D13FA1F03FC0D33FF9F0D43F39F13AC02C
:1042C000112341F0053008F04DC08C2F8F710E94F2
:1042D0005E2648C0063008F045C0F7CF112339F0FC
:1042E0008C2F8F710E9418263DC01123C9F38C2F8B
:1042F0008F710E94392636C0112329F08C2F8F71BF
:104300000E9403262FC00E94FE252CC0112349F0D5
:10431000CF718C2F0E94182663E08C2F0E940628F4
:1043200021C081E00E941B280230E0F082E00E9460
:104330001B2818C0112331F0002391F28D2F0E9409
:10434000371F10C0002399F2D93349F41FEF23EF30
:1043500031E0115020403040E1F700C000008D2FC7
:104360000E94851F88EF8C0D843020F40E94AE1DC2
:104370000E94BE14DD20C9F00E94852780FD15C073
:10438000F70112820E947F270E941826C7010E940F
:10439000F6210E947F27DF91CF911F910F91FF900F
:1043A000EF90DF90CF900C943926DF91CF911F9141
:1043B0000F91FF90EF90DF90CF9008950F931F9390
:1043C000CF93DF93EC01688179818A810E945C2719
:1043D0008C010E94B5260E94A625B801CE010E943C
:1043E000D21FDF91CF911F910F910895CF93DF934B
:1043F000EC01988189812B813C81232B31F08F3F07
:1044000031F481E09F3F19F403C081E001C080E0F6
:1044100080FD19C0CE010E94581481110CC00E9469
:104420008927882381F08A81882369F082E0DF91DF
:10443000CF910C941B28CE010E94DE21CE01DF918A
:10444000CF910C941313DF91CF9108950E94B02760
:104450000E94B3270E94D12780E090E00E940E1EA8
:1044600080E090E00C94241E809108019091090155
:104470000E9437290C9426220E94A0270C943422F3
:10448000E92FE295EF704E2F50E0FA013297EE30AF
:10449000F105B0F4EB58FF4F0C94CE32803F91F011
:1044A00018F4883E68F40EC0843F51F40BC0883E77
:1044B00048F0813F29F406C093FB882780F90895CE
:1044C00080E0089581E008950E9451270E944022D3
:1044D0000895CF93DF9300D000D01F92CDB7DEB701
:1044E0000F900F900F900F900F90DF91CF91089544
:1044F000CF93DF9300D000D000D0CDB7DEB72696A3
:104500000FB6F894DEBF0FBECDBFDF91CF910895F7
:104510001F93CF93DF93C091C20116E08091C30136
:10452000C81799F0D0E01C9FF0011D9FF00D1124D9
:10453000EC53FE4F4081518162817381848195816A
:104540000E9478222196C770E9CFDF91CF911F9109
:1045500008954091F4015091F5016091F601709138
:10456000F7018091F8019091F9010C9478220F9352
:104570001F93CF93DF938091F90182958F7009F09B
:104580005DC08091F601882309F458C08091C20172
:104590001091C3016091F4017091F501C091F70190
:1045A000D091F80191E06F3F09F090E0292F06E0EB
:1045B000811709F443C0209721F07F3F21F030E0BC
:1045C00003C031E001C0322F90E030FD34C0089FBD
:1045D000F001099FF00D1124DF01AC53BE4F11967D
:1045E0003C911197371327C03C91361324C0129683
:1045F0003C91129731111FC013964D915C91149705
:104600004C1B5D0B483C5105B0F48091F9018F7053
:1046100080618093F901E753FE4F80818F70806144
:10462000808384EF91E00E94F621DF91CF911F916A
:104630000F910C94882201968770BACFDF91CF91A9
:104640001F910F9108959F92AF92BF92CF92DF92E8
:10465000EF92FF920F931F93CF93DF93CDB7DEB707
:1046600061970FB6F894DEBF0FBECDBF8C0185E019
:10467000F801DE011D9601900D928A95E1F7F8018F
:1046800040815181E2809091F4016091F501209187
:10469000F7013091F8012115310531F06F3F31F408
:1046A00081E09F3F19F403C081E001C080E0F82F52
:1046B000F1709F2E80FD46C1F801A380B48084EF85
:1046C000C82E81E0D82EF090F601F501E21BF30B25
:1046D000FF2009F4DFC08091F901E83CF10508F002
:1046E0009BC0282F207F09F052C0561313C04913D6
:1046F00011C0FE2CE1100EC08F7080618093F90113
:104700000E94A922C6010E94F6218091F901F801B8
:10471000858358C1AB2831F05F3F31F481E04F3FD2
:1047200019F403C081E001C080E080FD03C081E096
:104730008E2502C080E090E0F82FF170FF2E80FF00
:104740001CC08091C2012091C30136E0821709F498
:1047500017C190E0389FF001399FF00D1124EC5300
:10476000FE4F6181561306C06081461303C062810B
:10477000E61203C001968770E9CFFE2CEE2009F403
:1047800021C18091F90181608093F9015AC05613CB
:1047900006C0491304C0E11002C0F8019FC04D8754
:1047A0005E878D859E850E946422882379F1EE20A4
:1047B00069F12091F901822F82958F7090E0029724
:1047C00074F08091F4019091F50198878F83198698
:1047D000BB86AA862C87CE0107960E94F62186E02A
:1047E000F801A4EFB1E001900D928A95E1F70E94E3
:1047F000B7220E94A9220DC0561729F14D875E8766
:104800008D859E850E94642281112CC0C8010E9462
:10481000F621FF24F394D6C0282F207F69F77A2D44
:10482000B98AA88A6E2D89890E94692284EF91E055
:104830000E94F62186E0F60111928A95E9F70E941E
:10484000A922F12CBFC04913D9CFE110D7CFF8016D
:104850008583C8010E94F62186E0F60111928A95AF
:10486000E9F7B0C0EE2091F22091F901822F8295F4
:104870008F7090E002970CF4B2CF8091F401909188
:10488000F5019A8389831B82BD82AC822E83CE017F
:104890000196A3CFE83CF10508F047C0FE2CEE20BE
:1048A00009F4B4CF561330C049132EC02091F9013A
:1048B00020FD21C0822F82958F70482F50E0411536
:1048C0005105C9F0F80125834F30510541F08F5F44
:1048D000982F9295907F822F8F70892B8583C801A6
:1048E0000E94F62186E0F801A4EFB1E001900D925C
:1048F0008A95E1F742C086E0F801A4EFB1E00190AB
:104900000D928A95E1F75EC04D875E878D859E8505
:104910000E946422811163CF8091F90181608093AC
:10492000F901C8010E94F6214DC07A2DB98AA88AE2
:104930006E2D89890E94692286E0F60111928A957E
:10494000E9F71BC0EE2009F461CF4D875E878D85A6
:104950009E850E946422F82E882309F457CF86E0B2
:10496000F801A4EFB1E001900D928A95E1F784EF90
:1049700091E00E94311F0E94B7220E94A92222C00A
:104980004D875E878D859E850E945127292F229510
:104990002F70223028F49F7039F0811105C00BC0B0
:1049A000243028F49F7049F4805E883020F0C801DC
:1049B0000E94F6219F2CF92C05C0F8019581907F6B
:1049C00099F7F9CF8F2D61960FB6F894DEBF0FBE21
:1049D000CDBFDF91CF911F910F91FF90EF90DF90AE
:1049E000CF90BF90AF909F90089588EC90E008958D
:1049F0001F93CF93DF93CDB7DEB72C970FB6F89404
:104A0000DEBF0FBECDBF4F83588769877A878B87FC
:104A10009C87CE0107960E9423238823D1F09F8193
:104A200088852A853B85232B31F08F3F31F481E047
:104A30009F3F19F403C081E001C080E080FD47C0C2
:104A40004F81588569857A858B859C850E9478225F
:104A50003EC086E0FE013796DE01119601900D9270
:104A60008A95E1F7FF81E8856A857B856115710587
:104A700031F0EF3F31F481E0FF3F19F403C081E0F2
:104A800001C080E080FD23C02091C30130E0C90156
:104A90000196877099274091C20150E084179507CD
:104AA000F1F1F983EA837D836C8396E0929FD001D4
:104AB000939FB00D1124AC53BE4FFE01319601906F
:104AC0000D929A95E1F78093C3010E94882216E027
:104AD0008091C2019091C301891771F1189FC001A3
:104AE00011248C539E4F0E942323882329F1E091A7
:104AF000C2011E9FF0011124EC53FE4F40815181F1
:104B000062817381848195810E9478228091C201A3
:104B100090E00196877099278093C201D9CF0E94B7
:104B20003C221092C3011092C201E4EFF1E086E052
:104B3000DF011D928A95E9F72C960FB6F894DEBF37
:104B40000FBECDBFDF91CF911F91089508950895B5
:104B50000C94A7250C94A8250E94AA256093030213
:104B60007093040280930502909306020C9426220F
:104B70000C94AC250F931F93009103021091040233
:104B80002091050230910602602B712B822B932B12
:104B90001F910F910C94AC250F931F93009103026A
:104BA00010910402209105023091060260237123C6
:104BB000822393231F910F910C94AC250F931F9385
:104BC0000091030210910402209105023091060227
:104BD00060277127822793271F910F910C94AC2592
:104BE0000C94A7250E94F0256093FF0170930002AA
:104BF00080930102909302020C94262260E070E000
:104C0000CB010C94F2250F931F9341E050E060E03C
:104C100070E08A019B0104C0000F111F221F331F87
:104C20008A95D2F7C901B8011F910F910C94F22512
:104C30000F931F9341E050E060E070E004C0440F28
:104C4000551F661F771F8A95D2F78091FF019091BB
:104C50000002A0910102B09102028A019B01082B7F
:104C6000192B2A2B3B2BC901B8011F910F910C94D2
:104C7000F2250F931F9341E050E060E070E004C024
:104C8000440F551F661F771F8A95D2F740955095A0
:104C9000609570958091FF0190910002A0910102B2
:104CA000B09102028A019B01082319232A233B2386
:104CB000C901B8011F910F910C94F2250F931F9316
:104CC00041E050E060E070E004C0440F551F661FF3
:104CD000771F8A95D2F78091FF0190910002A091F1
:104CE0000102B09102028A019B01082719272A2795
:104CF0003B27C901B8011F910F910C94F2250F9326
:104D00001F930091FF011091000220910102309148
:104D10000202602B712B822B932B1F910F910C940D
:104D2000F2250F931F930091FF0110910002209133
:104D300001023091020260237123822393231F9189
:104D40000F910C94F2250F931F930091FF01109186
:104D50000002209101023091020260277127822710
:104D600093271F910F910C94F225089524E0929FB0
:104D7000900D1124890FE82FE695E695E69587704A
:104D800051E001C0550F8A95EAF785E0E89FF001F0
:104D90001124E650FE4F20E030E070E04081CB016E
:104DA000022E02C0969587950A94E2F7817081954C
:104DB00084278523842781932F5F3F4F253031053A
:104DC00069F7089524E0929F900D1124890F682FB0
:104DD000669566956695982F977085E0689FB001F7
:104DE000112440E050E080E0FB01E40FF51FE650A5
:104DF000FE4F208130E0092E02C0369527950A9497
:104E0000E2F721703327042E01C0220F0A94EAF73B
:104E1000822B4F5F5F4F4530510531F70895BF92A8
:104E2000CF92DF92EF92FF920F931F93CF93DF9376
:104E30008C01C090FF01D0900002E0900102F09040
:104E400002028091030290910402A0910502B091A8
:104E50000602C82AD92AEA2AFB2ACFE1D0E0D701E4
:104E6000C6010C2E04C0B695A795979587950A9410
:104E7000D2F780FD04C0219790F7B12C07C0BC2E5B
:104E8000B8018C2F0E94C7140197A9F38B2DDF91D5
:104E9000CF911F910F91FF90EF90DF90CF90BF9037
:104EA0000895CF93DF93EC010E940F27BE010E946B
:104EB000C714DF91CF9108951F93CF93DF93EB0138
:104EC0009091C101992321F0CB010E94512713C079
:104ED000882349F0CB010E940F27182F682FCE019D
:104EE0000E94B62604C0CB010E94E226182FBE0104
:104EF000812F0E94C714DF91CF911F910895809157
:104F0000070285958595859508958091070287709C
:104F1000089590910702977081E009F480E0089568
:104F200080911302089590911302892B80931302AC
:104F30000895809590911302892380931302089518
:104F400010921302089590911202892B80931202FD
:104F500008958095909112028923809312020895FA
:104F60001092120208951092110208958091080281
:104F7000089508950C94B9270C94BA2790910802CB
:104F8000981721F0809308020C94BC270895809113
:104F90000802882329F01092080280E00C94BC27B4
:104FA0000895E0910801F091090180911302808336
:104FB000E0910801F0910901908180911202892B02
:104FC0008083E0910801F0910901908180911102A4
:104FD000892B808380910802882381F0E091080169
:104FE000F09109019081892B808380910801909133
:104FF00009010E94F12881110E94C72780910801B0
:10500000909109010C94BA1D0C94B92798E0899FDE
:1050100090011124262B209307020E9418268091CC
:1050200007028595859585950C94042810920702B2
:1050300080E00C94042820910702809582238093BD
:105040000702982F977079F430E0482F082E000C53
:10505000550B2417350739F08595859585950E9460
:1050600039260C94162808959093A1018093A001ED
:1050700008958295982F937344E0949F9001112492
:105080008C7C86958695282B822F8575880F2A7AA9
:105090002695822B08956FEF7FEF80E090E00C94CF
:1050A0000D3380E090E00E94E93221E08C3E9E4F7B
:1050B00009F020E0822F089582E090E00C94DB322A
:1050C00083E090E00C94DB32CF9384E090E00E9488
:1050D000DB32C82F81E290E00E94DB322C2F30E0DF
:1050E000A901582BCA01CF910895CF93C92F682FDA
:1050F00084E090E00E94EF326C2F81E290E0CF914B
:105100000C94EF328FE090E00C94E332AB01BC01E1
:105110008FE090E00C9401336CEE7EEF80E090E045
:105120000E940D3360E082E090E00E94EF3260E088
:1051300083E090E00E94EF3210920302109204028A
:10514000109205021092060260E084E090E00E9456
:10515000EF3260E081E290E00E94EF3260E085E0B3
:1051600090E00E94EF3260E086E090E00E94EF3233
:105170006FEF87E090E00E94EF3240E050E0BA012C
:1051800088E090E00E94013360E08DE090E00E94B2
:10519000EF3240E050E0BA0188E190E00E94013334
:1051A00060E087E190E00E94EF3240E050E0BA0119
:1051B0008CE190E00E94013360E080E290E00E9488
:1051C000EF3240E050E0BA0188E190E00E94013304
:1051D0000C94A6120C948C28682F8EE090E00C940E
:1051E000EF32FC01329697E080E0915029F0219156
:1051F0002223D9F38F5FF9CF0895662349F0FC018C
:10520000329608962191621729F0E817F907D1F72D
:1052100080E0089581E008959C01FC0132969FEFA3
:1052200080E04191461789F09F3F19F4411101C078
:10523000982F8F5F8630A9F79F3F39F0F901E90F6A
:10524000F11D97FDFA956283089508959C012A5FE8
:105250003F4FFC014281461301C012820196821722
:105260009307B9F708950C940C290C9426290296FB
:1052700026E0FC0111922A95E9F7089508950C940F
:105280003E290C943E290E9441290E94F2160E9458
:105290003F2980E00E948F1691E0811101C090E0CB
:1052A000892F08950C943E290C9452290E94542968
:1052B00080914A03843049F11092150220E488E17C
:1052C00090E00FB6F894A895809360000FBE2093ED
:1052D000600080E00E94BE140E94542983B7817F41
:1052E000846083BF83B7816083BF7894889583B7D8
:1052F0008E7F83BF0FB6F894A89580916000886177
:1053000080936000109260000FBE08950C943E29B7
:105310000E943C220E94AE1D0E94BE140C9486295D
:105320001F920F920FB60F9211248F939F93AF93FA
:10533000BF9380911502811113C080914003909119
:105340004103A0914203B09143034196A11DB11DB9
:105350008093400390934103A0934203B09343038F
:10536000BF91AF919F918F910F900FBE0F901F90A3
:10537000189582E084BD93E095BD9DE797BD80932D
:105380006E0008952FB7F8948091400390914103E7
:10539000A0914203B09143032FBF08952FB7F89413
:1053A00060914003709141038091420390914303C7
:1053B0002FBF08959C014FB7F894809140039091BE
:1053C0004103A0914203B09143034FBF821B930B53
:1053D000089578941F920F920FB60F9211248F9315
:1053E0009F93AF93BF938091400390914103A0910D
:1053F0004203B09143030196A11DB11D8093400368
:1054000090934103A0934203B0934303BF91AF91A4
:105410009F918F910F900FBE0F901F90189581E074
:105420008093E00080E28093D8001092C9008FE062
:1054300097E20197F1F700C0000087E090EBDC01F4
:105440008093530390935403A0935503B093560352
:105450009CE088E10FB6F894A895809360000FBE99
:1054600090936000FFCF0C94E6170E94F2168FE134
:105470009EE40197F1F700C000000E94F21680E060
:105480000E948F1683FF04C00E94332A0C940F2AB7
:1054900008950E945128811102C00E94EA280E94AA
:1054A0005C28809314020E946428909345038093A3
:1054B00044030E946028682F70E080E090E00E9422
:1054C000B8256091FF0170910002809101029091D6
:1054D00002020C94F0258091210208959FB7F89460
:1054E000109218029FBF90914A03943009F057C060
:1054F0009091E9009F703091EC00232F217030FDD6
:1055000020E8922B26E02093E9002091EB0020FF79
:1055100043C02091EE0027FF3FC0209116022223B6
:1055200021F02091E80025FF37C01092160226E0F6
:105530003091E80035FD15C030914A03343061F5F3
:105540003091EB0035FD28C0215021F481E080939B
:10555000160222C0EFECF7E03197F1F700C000002F
:10556000E7CF8093F1008091E80085FD0AC080912B
:10557000E80080FFFCCF8091E8008E778093E80000
:1055800006C08FB7F89421E0209318028FBF9F7058
:105590009093E90080E008959F709093E9008FEF69
:1055A0000895CF93DF9300D01F92CDB7DEB79091CF
:1055B0004A03943019F589837B836A8385E080935D
:1055C000E9008FEF9091E800815095FD06C09AE6C2
:1055D0009A95F1F700C08111F5CF8091E80085FF21
:1055E0000DC040E050E063E070E0CE0101960E9403
:1055F000B52D8091E8008E778093E8000F900F9092
:105600000F90DF91CF910895BC0184E00C94D12AD2
:10561000BC0183E00C94D12A22E02093E9002FEF13
:105620003091E800215035FD06C03AE63A95F1F791
:1056300000C02111F5CF2091E80025FF0BC040E00C
:1056400050E065E070E00E94B52D8091E8008E7713
:105650008093E8000895CF93DF9321E02093E90041
:105660002FEF3091E800215035FD06C03AE63A951B
:10567000F1F700C02111F5CF2091E80025FF14C0FB
:10568000EC0140E050E068E070E00E94B52D8091B0
:10569000E8008E778093E80088E0FE01A9E1B2E09F
:1056A00001900D928A95E1F7DF91CF910895CF9304
:1056B000603219F520914A032430F9F4C091E900D1
:1056C000CF703091EC00232F217030FD20E8C22BE9
:1056D00023E02093E9002091E80020FF0BC040E088
:1056E00050E060E270E00E94B52D8091E8008E7776
:1056F0008093E800CF70C093E900CF9108958BE4C8
:1057000093E10E94EB0A80914903811109C00E9434
:10571000912F0E94EE2F8091E20084608093E2003E
:10572000089587E493E10E94EB0A109249030895DB
:1057300083E493E10C94EB0A8FE393E10C94EB0A7E
:105740008BE393E10E94EB0A0C94882920911702C5
:105750002F5F822F62E30E949A32992319F02093DF
:10576000170208951092170280911802882371F190
:1057700080914A03843041F58091E9008F70209137
:10578000EC00922F917020FD90E8892B96E0909389
:10579000E9009091EB0090FF14C09091EE0097FF0C
:1057A00010C09091E80095FF03C01092F100F9CF6E
:1057B0009091E80090FF05C09091E8009E7790934B
:1057C000E8008F708093E90010921802089542E07B
:1057D00061EC81E00E940A2F42E061EC82E00E94CD
:1057E0000A2F42E261EC85E00E940A2F42E261EC5E
:1057F00083E00E940A2F42E260EC84E00E940A2FBC
:1058000042E261EC86E00C940A2F80914C038330D5
:1058100009F462C030F4813071F0823009F49BC029
:1058200008958A3009F487C08B3009F46DC089303F
:1058300009F0A9C020C080914B03813A09F0A3C0B0
:105840008091E800877F8093E80080914F039091DA
:105850005003892B21F468E089E192E003C060E005
:1058600080E090E070E00E944B2E8091E8008B7702
:105870008093E800089580914B03813209F083C042
:1058800080914F0390915003009719F0039709F00E
:105890007AC08091E800877F8093E8008091E800DB
:1058A00082FD05C080914A038111F8CF6CC0209120
:1058B000F3008091F20090E0922B029729F48091FE
:1058C000F1008B7F813021F48091F10080932102DF
:1058D0008091E8008B7753C080914B03813A09F0A7
:1058E00052C080914F0390915003892B09F04BC017
:1058F0008091E800877F8093E8008091E80080FF36
:10590000FCCF8091140136C080914B038132D9F5D0
:1059100080914F0390915003892BA9F58091E80065
:10592000877F8093E8000E943F2F80914D038093F2
:1059300014010C943C2280914B03813221F580911B
:10594000E800877F8093E8000E943F2F80914E03FC
:1059500080932202089580914B03813AA1F48091B3
:10596000E800877F8093E8008091E80080FFFCCF0B
:10597000809122028093F1008091E8008E778093DD
:10598000E8000C943F2F0895CF93DF93CDB7DEB797
:10599000A0970FB6F894DEBF0FBECDBF84B7877F48
:1059A00084BF0FB6F894A8958091600088618093B9
:1059B0006000109260000FBE90E080E80FB6F8948F
:1059C00080936100909361000FBE0E944E1E0E9462
:1059D000912F0E94EE2F8091E20084608093E2007C
:1059E0008EE69AE20E94342878940E947F320E94C8
:1059F000541E8AE091E00E94A91D8AE293E10E9470
:105A0000EB0A80914A03853089F486E293E10E9493
:105A1000EB0A0E94562980914803882391F30E9443
:105A20004329882371F30E94A02DEBCF0E94881E8A
:105A300080914A03843009F58093E9008091E80061
:105A400082FF1BC08091E80085FF0AC040E050E063
:105A500060E270E0CE0101960E94002E91E001C04C
:105A600090E08091E8008B778093E800992329F0FB
:105A700060E2CE0101960E9448180E94461E0E94D4
:105A8000451EBFCF0C94442D292F332723303105D9
:105A9000C9F060F42130310581F02230310509F080
:105AA00047C084E990E023E833E146C02132310564
:105AB00011F12232310561F13BC082E190E027E132
:105AC00034E13AC099278130910561F040F082308D
:105AD000910559F0039761F5EFE4F3E108C0EFE7B2
:105AE000F3E105C0EBE6F3E102C0E5E5F3E1849103
:105AF00090E09F0121C065307105D0F4660F771FDB
:105B0000FB01EA56FE4F2081318189E090E014C00C
:105B10006530710568F4FB01EE0FFF1FE457FE4F7F
:105B200020813181FB01E957FE4F808190E004C064
:105B300080E090E020E030E0FA0131832083089596
:105B400019BC82E089BD09B400FEFDCF8091D80068
:105B50008F7D8093D8008091E00082608093E00088
:105B60008091E00081FDFCCF0895CF92DF92EF920B
:105B7000FF920F931F93CF93DF93EC018B017A0178
:105B80000E945E2F811133C0E114F10439F0F70156
:105B900080819181081B190BC80FD91FC12CD12CF2
:105BA0000115110519F18091E80085FD16C080915D
:105BB000E8008E778093E800E114F10449F0F701E2
:105BC00080819181C80ED91ED182C08285E00FC02C
:105BD0000E945E2F882321F30AC089918093F100EF
:105BE00001501109FFEFCF1ADF0ADACF80E0DF9111
:105BF000CF911F910F91FF90EF90DF90CF9008957C
:105C0000CF92DF92EF92FF920F931F93CF93DF9388
:105C1000EC018B017A010E945E2F811133C0E114E7
:105C2000F10439F0F70180819181081B190BC80F2D
:105C3000D91FC12CD12C0115110519F18091E80053
:105C400085FD16C08091E8008B778093E800E11411
:105C5000F10449F0F70180819181C80ED91ED182EB
:105C6000C08285E00FC00E945E2F882321F30AC006
:105C70008091F100899301501109FFEFCF1ADF0ADB
:105C8000DACF80E0DF91CF911F910F91FF90EF90DD
:105C9000DF90CF9008952091510330915203261741
:105CA000370748F06115710539F42091E8002E7727
:105CB0002093E80001C0B901FC0120E061157105E5
:105CC00079F180914A038823F1F18530F1F18091D7
:105CD000E80083FD3CC08091E80082FD2EC08091E9
:105CE000E80080FFEBCF2091F3008091F20090E07C
:105CF000922B6115710551F08830910538F421918E
:105D00002093F100615071090196F3CF21E00897CB
:105D100009F020E08091E8008E778093E800CECFF4
:105D20002111CFCF0AC080914A03882361F08530CA
:105D300061F08091E80083FD0AC08091E80082FF55
:105D4000F2CF80E0089582E0089583E0089581E035
:105D5000089520915103309152032617370748F0D8
:105D60006115710539F42091E8002E772093E80041
:105D700001C0B901FC0120E06115710591F180912C
:105D80004A03882309F440C0853009F43FC080915C
:105D9000E80083FD3DC08091E80082FD2FC0809126
:105DA000E80080FFE9CF2091F3008091F20090E0BD
:105DB000922B6115710559F08830910540F42491BA
:105DC0002093F1003196615071090196F2CF21E0E4
:105DD000089709F020E08091E8008E778093E80032
:105DE000CBCF2111CCCF0AC080914A03882361F028
:105DF000853061F08091E80083FD0AC08091E80061
:105E000082FFF2CF80E0089582E0089583E0089554
:105E100081E00895982F973068F59093E9009817DE
:105E200039F07091EC002091ED005091F00003C02A
:105E3000242F762F50E021FD02C09F5FECCF3091E0
:105E4000EB003E7F3093EB003091ED003D7F3093CF
:105E5000ED003091EB0031603093EB007093EC007B
:105E60002093ED005093F0002091EE0027FDE5CF48
:105E700080E008958F708093E90081E0089580911B
:105E80004B0387FF11C08091E80082FD05C080911F
:105E90004A038111F8CF11C08091E8008B770BC0C5
:105EA00080914A03882349F08091E80080FFF8CF71
:105EB0008091E8008E778093E80008952091E400B7
:105EC0003091E50095E64091EC00842F817040FF11
:105ED00023C08091E80080FD1DC080914A03882383
:105EE00099F0853099F08091EB0085FD11C04091CB
:105EF000E4005091E5002417350729F3915011F083
:105F00009A01E1CF84E0089582E0089583E0089546
:105F100081E0089580E008954091E80042FFDDCFE0
:105F200008950E94FF2F0E940730E0EEF0E080818C
:105F300081608083E8EDF0E080818F77808319BCF9
:105F4000A7EDB0E08C918E7F8C9380818F7E8083D3
:105F50001092490308950F931F93CF93DF930E94EC
:105F6000FF2F0E940730C8EDD0E088818F778883AB
:105F700088818068888388818F7D888319BC10928E
:105F80004A0310924603109248031092470300EE12
:105F900010E0F80180818B7F808388818160888315
:105FA00042E060E080E00E940A2FE1EEF0E08081B4
:105FB0008E7F8083E2EEF0E080818160808380814B
:105FC00088608083F80180818E7F808388818061F2
:105FD0008883DF91CF911F910F910895E8EDF0E054
:105FE00080818F7E8083E7EDF0E080818160808317
:105FF00084E082BF81E0809349030C94AB2FE8EDED
:10600000F0E080818E7F80831092E20008951092EC
:10601000DA001092E10008951F920F920FB60F92CE
:1060200011242F933F934F935F936F937F938F939D
:106030009F93AF93BF93EF93FF938091E10082FF13
:106040000BC08091E20082FF07C08091E1008B7F4E
:106050008093E1000E94A62B8091DA0080FF1DC092
:106060008091D80080FF19C08091DA008E7F8093E4
:10607000DA008091D90019BC80FF0BC082E089BD95
:1060800009B400FEFDCF81E080934A030E947F2B7C
:1060900004C010924A030E94912B8091E10080FF7E
:1060A00019C08091E20080FF15C08091E2008E7FD0
:1060B0008093E2008091E20080618093E200809111
:1060C000D80080628093D80019BC85E080934A0391
:1060D0000E949C2B8091E10084FF2FC08091E20000
:1060E00084FF2BC019BC82E089BD09B400FEFDCF3E
:1060F0008091D8008F7D8093D8008091E1008F7EC1
:106100008093E1008091E2008F7E8093E200809195
:10611000E20081608093E20080914603882311F0C1
:1061200084E007C08091E30087FD02C081E001C0E8
:1061300083E080934A030E94A02B8091E10083FFBB
:1061400029C08091E20083FF25C08091E100877F14
:106150008093E10082E080934A031092460380918D
:10616000E1008E7F8093E1008091E2008E7F80933A
:10617000E2008091E20080618093E20042E060E012
:1061800080E00E940A2F8091F00088608093F000E8
:106190000E94982BFF91EF91BF91AF919F918F91AA
:1061A0007F916F915F914F913F912F910F900FBE13
:1061B0000F901F9018951F920F920FB60F921124F7
:1061C0002F933F934F935F936F937F938F939F93FF
:1061D000AF93BF93CF93DF93EF93FF93C091E90009
:1061E000CF708091EC00D82FD17080FDD0E8109254
:1061F000E9008091F000877F8093F00078940E94FE
:106200001F311092E9008091F00088608093F000C7
:10621000CD2BCF70C093E900FF91EF91DF91CF912B
:10622000BF91AF919F918F917F916F915F914F91AE
:106230003F912F910F900FBE0F901F9018951F93B5
:10624000CF93DF93CDB7DEB7AA970FB6F894DEBF32
:106250000FBECDBFEBE4F3E08091F100819323E02A
:10626000E335F207C9F70E94052C8091E80083FF0F
:106270002EC180914B0390914C03492F50E04A303E
:10628000510508F024C1FA01ED57FF4F0C94CE32AE
:10629000803821F0823809F01AC108C08091470384
:1062A00090914803992389F082600FC080914F0339
:1062B0008F70873008F00BC18093E9008091EB006C
:1062C00085FB882780F91092E9009091E800977F7C
:1062D0009093E8008093F1001092F100D1C0282F34
:1062E0002D7F09F0F4C0882319F0823061F0EFC0EF
:1062F00080914D03813009F0EAC0933009F080E0CD
:10630000809348032EC080914D0381112AC0809153
:106310004F038F702FEF280F263008F0D8C08093DE
:10632000E9002091EB0020FF1CC0933021F4809104
:10633000EB00806214C09091EB0090619093EB00B1
:1063400021E030E0A90102C0440F551F8A95E2F711
:106350004093EA001092EA008091EB0088608093FD
:10636000EB001092E9008091E800877F8093E800BD
:106370000E943F2FACC08111AAC010914D031F771E
:106380008091E3008078812B8093E3008091E80086
:10639000877F8093E8000E943F2F8091E80080FF74
:1063A000FCCF8091E30080688093E300111102C06C
:1063B00082E001C083E080934A0389C08058823024
:1063C00008F085C080914D0390914E038C3D53E0C1
:1063D000950779F583E08A838AE289834FB7F89439
:1063E000DE01139620E03EE051E2E32FF0E050930F
:1063F0005700E49120FF03C0E295EF703F5FEF701C
:106400008E2F90E0EA3010F0C79601C0C0968D93B1
:106410009D932F5F243149F74FBF8091E800877F1C
:106420008093E8006AE270E0CE0101960E944B2E54
:1064300016C060914F0370915003AE014F5F5F4FE4
:106440000E94422DBC01892B09F441C09091E800C3
:10645000977F9093E80089819A810E94A92E80916C
:10646000E8008B778093E80032C0803881F5809116
:10647000E800877F8093E800809146038093F100D5
:106480008091E8008E7772CF811121C080914D03F9
:1064900090914E0399270297D4F48091E800877F6A
:1064A0008093E80080914D03809346030E943F2F24
:1064B00080914603811106C08091E30087FD02C0F0
:1064C00081E001C084E080934A030E94E72B809121
:1064D000E80083FF0AC08091E800877F8093E8008E
:1064E0008091EB0080628093EB00AA960FB6F8943F
:1064F000DEBF0FBECDBFDF91CF911F910895CF9327
:1065000080914A038823A1F0C091E900CF70909157
:10651000EC00892F817090FD80E8C82B1092E90073
:106520008091E80083FD0E941F31CF70C093E90085
:10653000CF910895991B79E004C0991F961708F030
:10654000961B881F7A95C9F780950895AA1BBB1BD7
:1065500051E107C0AA1FBB1FA617B70710F0A61B63
:10656000B70B881F991F5A95A9F780959095BC0184
:10657000CD01089597FB072E16F4009407D077FD00
:1065800009D00E94A63207FC05D03EF49095819573
:106590009F4F0895709561957F4F0895EE0FFF1FEF
:1065A0000590F491E02D09946927962769277827AB
:1065B000872778270895F999FECF92BD81BDF89A73
:1065C000992780B50895A6E1B0E044E050E00C942E
:1065D0001533A8E1B0E042E050E00C941533262FCB
:1065E000F999FECF92BD81BDF89A019700B40216C9
:1065F00039F01FBA20BD0FB6F894FA9AF99A0FBE77
:1066000008950396272F0E94F0320E94EF32252F23
:106610000E94F032242F0C94F0320196272F0E9412
:10662000F0320C94EF32DC01CB01FC01F999FECF82
:1066300006C0F2BDE1BDF89A319600B40D9241500A
:0A6640005040B8F70895F894FFCF1A
:10664A00B0044006600940FF09026B2A2B2B0C2B71
:10665A00082B042B0191933436379667F6F5F3F736
:10666A00E200E900EA00B500B600B700CD008301F8
:10667A00CC008A01920194012102230224022502FC
:10668A00260227022A02B300B4006F00700081823A
:10669A00839492C63597E200E900EA00B500B60095
:1066AA00B700CD008301CC008A0192019401210236
:1066BA00230224022502260227022A02B300B4007A
:1066CA006F00700081828340224D3222EC144B14F9
:1066DA009F146D1429149513AE13CE13E7130014E7
:00000001FF
